:020000041100E9
:10300000F7B5164B0192C318021D002000938823C8
:103010005B05D3181B685C1C1AD09CB2402C18D8D6
:103020008D781E0CAC466746CD782D023D43AE42EE
:1030300006D1019800280ED110000C70240A4C70A3
:1030400003249BB20733A343D218009B9A42DED3DA
:10305000FEBD4432F9E71000FAE7C046FC0F00005D
:10306000802213B503000324019189B25201073174
:103070009B18A14304305A1A88235B05C3181B68A8
:10308000591C03D190429241104016BD99B240297B
:1030900007D80B000733A343C0189042ECD300209D
:1030A000F3E74430F9E7134B134A1B68126810B575
:1030B000F424934201D81A00F024104BA4021B6898
:1030C0009A4210D813000E4A12689A420ED3013366
:1030D00007D1F0239B029C4203D10A49054808F01E
:1030E00067FC200010BDF824A402ECE7FC24A40235
:1030F000F7E7C04600C0031100D0031100E0031140
:1031000000F00311FFFFFF7FF0B59BB015000490A6
:103110000391402A00D9A0E006AB59801A80FFF73E
:10312000C2FF0400042816D9002206A9FFF768FF91
:10313000052810D906AB1B88AB420CD1002D07D057
:10314000514B2A000499C01808F082FA002802D1D5
:1031500001201BB0F0BD06AB1D8020000699FFF7D3
:103160007FFF041E7BD1069B0793FFF79CFF802304
:103170005B01C61880230700DB029E4201D3F026C4
:10318000B60288235B05F31801931B68013302D054
:10319000019808F01DF93D49019808F009FC3B1D14
:1031A0000293331D05938822029B52059B181B68CE
:1031B00008935A1C3CD044219AB20091402A04D86A
:1031C0000320D11D814389B2009103991B0C8B42CE
:1031D00024D0402A22D80122300008A9FFF710FF8E
:1031E000021E1BD1380008A9FFF70AFF04000428BB
:1031F00031D9009A059B9B1880225201B218934244
:1032000040D288235B05C118009A09A808F000FB8A
:103210001D4B009A09A9F01808F042FA009A029B87
:103220009446634402931A4B029AFB189A42BAD30B
:1032300088235B05FC1821680198013908F0B8FB68
:10324000200008F0C5F8039A07AB5A8030000799B0
:10325000FFF706FF0400002C03D1002079E70428C3
:10326000FBD988235B05E018069908F0A1FB03232E
:10327000EA1C9A4300D16BE7034B0499E01808F06D
:103280000FFA65E70424ECE704000011FFFFFF7F5D
:10329000F80F0000F7B505001400402A21D80027D8
:1032A00001AE71803780FFF7FEFE042816D93A0080
:1032B0003100FFF7A5FE042810D93688BC420BD098
:1032C000BD4209D0221CB44200D9321C064B92B236
:1032D000C118280008F09CFA30B2FEBDC04300B20D
:1032E000FBE703204042F8E70400001137B5042251
:1032F00004000D0001A81649FFF7CCFF02000428C6
:103300000BD1019BA34208D3AB4204D0104901A8C2
:103310000195FFF7F9FE01203EBD0E4C2368200009
:10332000019308F055F8019920000139019108F046
:103330003FFB80235B01E418074B9C42EED1042243
:10334000034901A80195FFF7DFFE0020E4E7C0462E
:103350005555000000C003110000041130B589B0BC
:1033600008F0D6F910226946254808F039FB254BAC
:10337000009A9A420ED1019B029A0F2B33D800215A
:1033800001240698013B08D2002900D00292029B3A
:10339000013331D10023029325E0551CF2D1020004
:1033A0002100EFE710341022200004A908F018FBD8
:1033B000029B013301D1069B0293882304995B058C
:1033C000C918059B06981A03120B049105928142B5
:1033D00003D02B4201D108F01BFA019B013B019362
:1033E000019B002BDED1029B002B03D00493049899
:1033F0004168084709B030BDE025014C2D03EFE7D7
:1034000000000111504859368022F8B5964C974B70
:10341000D200002120001C6008F022F82300944A0A
:1034200088331A60934B1A786A23002A00D011332C
:10343000E3620A232365904B37221B780820A3639D
:103440008E4B2118E361102323628D4B3B25636172
:10345000C823DB00A36123008C331A602823013AC0
:10346000E26320646364CA67043A211DCA672100CD
:10347000BC310D602100C03108602100C4310B60F7
:1034800021000635CC310D602100083DC8310D60AA
:103490002100D0310A602200D43210602200D832DC
:1034A000136022000227E032210017604222DC3143
:1034B0000A6021001B3DE4310D602100E831086005
:1034C0002100EC310B6023000521F4331960230047
:1034D000F0331A602300183290331A6023009433BB
:1034E000186023001E3A98331A60AF23DB00236074
:1034F000644BFA262363644B644DE360644BF03104
:10350000A3642300FF31FC33B600A16021611E607B
:10351000A5627325E5656D3D6565A56596255D4AE2
:10352000AD00E264666258606766A56600270925FB
:10353000A767E566584F594D606720002567E26729
:103540003A6015279C30676007001A203860200019
:10355000A0300700212038602000A83007004C4828
:1035600038602000F830066026006427A4363760F3
:1035700026005F3FAC3637602600033FB036376029
:103580002600C637B436376026000027B8363760C5
:1035900038269E60424E96205E64424E5A66DE6138
:1035A000414E9A645E62F53EFF3E9E621E269A6719
:1035B000354A8000DE661F675F67DD651D6618623D
:1035C000DA67BE23394A5B00E250394BD8382350C2
:1035D00004302250C4225200A350C623E4205B00D2
:1035E000E1500433334AE1503349344BD16034491C
:1035F000800019503349E938FF38195032490430F6
:10360000195032493248D16132491163324951630C
:103610001900F4310860CE20304940001160304973
:10362000195019002F48F83108602F49D1658221BF
:103630002E4A89005A501A002D490832D1671A00C3
:103640002C49B432116088212B4A89005A501A0043
:103650002A49883211602A4ADA6408F081F9012087
:1036600007F06EFFF8BDC0460004FF1F8464FF1F13
:10367000506FFF1F2044FF1F4A0AFF1F3A07000038
:1036800080C3C9019A020000DC0500006A1800002E
:1036900050C3000088130000F009FF1F204E0000F7
:1036A0006509FF1F68100000C409000040420F00B8
:1036B00010270000FC00FF1F751CFF1F0000FF1FEC
:1036C000C92CFF1F5130FF1FE92EFF1F3520FF1FA0
:1036D0002527FF1F5120FF1FFD21FF1FC11FFF1FB7
:1036E0004929FF1F312AFF1F8D19FF1F5528FF1F72
:1036F0007925FF1F8525FF1FC11EFF1F791FFF1F93
:10370000391EFF1F0223F0B50124634D634E2B7059
:10371000634B8BB01C70634F039333680021092007
:103720007B7006F039FD092006F030FC031E05D140
:103730007A78552A02D0332A00D0A0E000233360E3
:10374000042006F0A3FE08F023F8FFF75DFE07F063
:1037500027FF1F2201240021534B1E261A70534BB2
:103760001C70534B1970534B19689143163A0A4316
:103770001A60602219689143403A0A431A6008F0BF
:10378000CFF807F0ADFE4C4B9847C120FF214B4BC3
:1037900080001A588A431A50C522920098588843CC
:1037A000BF39014399509858454908408021C901C3
:1037B0000143802099509958C0050902090A014324
:1037C000995080213F48490107F0EAFD0323220078
:1037D00000933D4901943D4808F0AAF816223C495F
:1037E00004A808F015F802AB04ACF618617820784C
:1037F000023406F0EBFBA642F8D1364C032001213F
:1038000006F0F8FC2268344B03201A40A023DB02A8
:1038100013432360802322689B04134323602268A0
:103820002E4B1A4080239B03134323602C4A2D4BBD
:10383000934200D8012007F02BFF07F049FE8023B8
:103840002268DB0413432360287807F099FE039B6A
:103850001878C0B207F09CFD07F08AFE22490420C8
:1038600007F0E6FD06F0DEFD00F040F800F08EFD0A
:1038700000F036FE00F0B8FB00200BB0F0BD009069
:103880002100194A042008F0B3F88023DB059C626C
:10389000FFF764FD54E7C0464A0AFF1F34F00040BA
:1038A0002044FF1F2862FF1F480AFF1F490AFF1F0D
:1038B000680AFF1FBCF00040E1A2000000E100E048
:1038C000FF00FFFF2444FF1FA856FF1F2454FF1FC3
:1038D00010BA001114F00040FF7FF8FFFFFF9FFFB8
:1038E0000080FF1F506FFF1F3B000108002210B532
:1038F0001100112007F0ACFD10BD0000F8B5002349
:103900000926374F374C3B62E3681120B343E3602D
:1039100007F0D6FF112007F073FE112007F078FEA4
:103920004023226880251343236080236268DB02E2
:1039300013436360A3682C4A2B43A360A36802214E
:103940001340A3608023A2689B0113431022A3604D
:10395000236C072093432364236C0F3A134323649F
:1039600080235B003B62226B204B1A402263626B18
:103970001A406263A26B1A40A263E26B1340E363D6
:10398000E3681B4A1340E36006F020FB0121072097
:1039900006F030FC174B11205A6C15435D6407F09C
:1039A0000FFFFD21144B154A89005A508023C72070
:1039B000626B5B0313436363E36880003343E3603C
:1039C0000F4B104A19581140802212020A431A5014
:1039D000802292051A6008220B4B5A63F8BDC0463C
:1039E00000F000403CF00040FFFFDFFFEFFFEFFF83
:1039F000FFFF7FFF003800400000FF1F5118FF1F2E
:103A000000E100E0FF00FFFF0000054007B50422D1
:103A1000044901A807F0FCFE012101A807F0A0FE5F
:103A200007BDC04626BA001170B52B4C238C002B65
:103A30002AD0FA22D200934201D2FFF7E7FF228A6E
:103A4000238C002A21D1DA0023826382A382E382BD
:103A500023836383A383E38322606260A260E260C6
:103A60001E4D1F4A6420EB8093420AD8FA220020A0
:103A7000D200934205D91B4A0A21981807F0D8FEB4
:103A8000C0B200232872238470BD0720E11CCA7FC6
:103A900001320240CA7705D10325201DC17F0131C3
:103AA0002940C17708325200A352002321001A0096
:103AB000088A01321B180231082AF9D1221DD27F4F
:103AC0009200A350626823689B18A2689B18E26862
:103AD0009B185B099BB2C3E72061FF1F0862FF1FB1
:103AE000B70B000030F8FFFF30B503A804880B20A7
:103AF000002C0ED14968074D087849780902014326
:103B00000A20A94205D1012120001980024B1B7A0D
:103B1000137030BD192A00000862FF1FF7B51500A9
:103B200008AA16884A680F4F147852781202224366
:103B30000A24BA4214D10122DBB2019200962A0073
:103B400007F0C0FB041E0BD1074B1B68002B07D0EE
:103B500068782A7800021043424250410130984769
:103B60002000FEBD022900004C61FF1F30B5012579
:103B700003790400BFB02B4211D00A49408806F0F7
:103B80000DFF28420BD0084B01A95B8D4D800B80A7
:103B9000064B00221B7A60880B7103F0DFFF3FB0F9
:103BA00030BDC0464461FF1FE040FF1F0862FF1F99
:103BB00010B50549054806F0A7FE0421044A05484A
:103BC00006F064FE10BDC0464461FF1FFFFF000009
:103BD0002CBA0011E040FF1F10B5024804F040FE6F
:103BE00010BDC0466D3B0011F0B593B005921D00AD
:103BF000DAB20F239B1ADFB20E239B1ADBB20493B7
:103C00001C9B049A023B5B08DB00134306AA13705B
:103C1000199E06AB2A0003900191581C059907F0E4
:103C2000F7FD3400002206AB013BBA4252D1002C12
:103C300000D0B9E0102221000AA807F011FC0AAB5D
:103C4000029306A91A78615C01344A401A70013364
:103C5000102CF6D10AAA1100019807F011FD2022BC
:103C6000212006AB9B18049A05991A7006AB2A000E
:103C7000C01807F0CDFD01350EAB58193A000021F0
:103C800007F0EEFB2F210123250006AA521813701E
:103C9000002E24D112AB3A003100D81B07F0E0FB14
:103CA000019806AA0EA907F0EBFC029B06AA925DFA
:103CB0001B7801365340029A1370130001330293AC
:103CC000102EF2D11C9A1B980AA907F0A1FD002022
:103CD00013B0F0BD01321C74D2B2240AA4E7340040
:103CE000102E00D92C00039B002B19D119002A009B
:103CF00006A807F0B5FB2200189906A807F088FD72
:103D0000039B0AAA06A81178185C01334140117080
:103D10000132102BF6D10AAA1100019807F0B0FC6D
:103D2000019806AA0EA907F0ABFC0023189A06A971
:103D3000C95CD25C4A401A99CA5401339C42F5D1FD
:103D4000039B012B19D11022002106A807F088FB44
:103D500022001A9906A807F05BFD00230AAA06A80C
:103D60001178185C0133414011700132102BF6D1EB
:103D70000AAA1100019807F083FC00221A9B361B47
:103D80001B191A93189B0EA91B191893BA4200D13C
:103D90007EE7CB7B01390133DBB20B74002B00D003
:103DA00076E70132D2B2F1E70120404290E700000D
:103DB00010B5134A134B5179134C19701179200027
:103DC0005970D17899709178D970517812781971A9
:103DD0005A712E2252429A712A32DA7145321A727F
:103DE0000A49313AFFF756FA102808D0102120006E
:103DF00007F01EFC102220000449FFF785F910BDD2
:103E00006509FF1F6061FF1F5061FF1F0DBC0000AF
:103E1000F0B5431805000020114F124A3E8889B0C2
:103E20000C00114956720792320A4A70320ECA705B
:103E300088701E70042639889870090A5970D870E5
:103E40009B19039301940D230849079A0496029540
:103E50000095FFF7C9FE0834E0B209B0F0BDC046D6
:103E60000862FF1F6061FF1F6961FF1F5061FF1F34
:103E7000012202700C4A0300117A41700C209870E4
:103E80009179D970D17919713A21597192789A71D1
:103E90003E22DA71054A117B1972517B5972917B6E
:103EA000D27B9972DA7270470862FF1F1462FF1F9B
:103EB00070B51F4A1F4BD17C04001B681E4A0029A5
:103EC00006D1190604D50323137000F039F870BD2C
:103ED00000211170022219002270013A627005322D
:103EE000A27010322271443A62712A32A2712432D5
:103EF0001140134210D0250041230835E3712800FA
:103F0000FFF7B6FF01002800FFF782FF0430C0B2C0
:103F1000E0700430C0B2DAE740232000E371074BC1
:103F200021721B880A306372FFF7A2FF0630EEE7AA
:103F30001462FF1F2C62FF1F2664FF1F0862FF1F11
:103F400010B5040006220E4907F062FC16220D4946
:103F5000E01D07F05DFC0C4B1B789B0963770B4B56
:103F60001A7A0023502A06D840333C2A03D840331B
:103F7000192A00D84033A37100231F20A37710BD56
:103F800044BA00118F61FF1F8961FF1F0862FF1F84
:103F900010B5142007F06CFC124B1422002118609D
:103FA00007F05EFA002007F05BFC012007F048FBF9
:103FB000022007F05DFA032003F0F6FE042005F06E
:103FC0000BFF052003F034F9062003F001FE072063
:103FD00001F05AF9082006F039FC092000F0CAFE69
:103FE00010BDC046A861FF1F07F082FB012007F04B
:103FF0004FFA07F085FB0000094B10B5040098420A
:1040000005D0012904D12000064906F07DFC10BD31
:104010000229FCD1013904F0E1FB0028F3D0F6E7D6
:10402000FEFF0000CE61FF1F70B50D7A100004AADC
:104030002C00168810221440154220D1002E20D1C9
:104040000A78022A18D14A68517815780E4A09026E
:104050002943914205D00D4A914209D01C800A247F
:1040600004E014220A491A8007F0D2FB200070BD38
:104070000C2208491A80F7E71C800124F6E708247F
:10408000F4E70B24F2E7C046F3FF0000F4FF000062
:10409000AC42FF1FE8BA001110B5040007490848F8
:1040A00006F032FC074804F01BFB0020E40704D5AF
:1040B0000721054A054806F0E9FB10BDCE61FF1F48
:1040C000FFFF0000F93F001174BA00112441FF1FE7
:1040D00000B50C4BBFB01A780B4902A800F0B0FA3B
:1040E0006B4680B2D880002809D06A46074B01A9E8
:1040F0001B889380064B0022188803F02FFD3FB0E9
:1041000000BDC046AC61FF1FAD61FF1F7E41FF1FB8
:104110008042FF1F00B50C4BBFB01A780B4902A8B4
:1041200001F076FB6B4680B2D880002809D06A4641
:10413000074B01A95B8D9380064B0022188803F082
:104140000DFD3FB000BDC046D661FF1FD761FF1F08
:104150002441FF1F8042FF1FF7B50E00377A1C0075
:1041600008AB11003D001A8820231D401F423CD19E
:104170003378022B3BD173681F785B781B023B437B
:104180001E4FBB4208D01E4FBB4214D01D4DAB4248
:1041900021D00A252800FEBD002A2AD1142C2AD8B5
:1041A0002200F06807F034FB174B1C70012CF1D98A
:1041B000FFF7B0FFEEE7002A1BD1202C1BD822000E
:1041C000F06807F025FB114B04211C70104B187888
:1041D00007F04EFADEE7E3B20124009201940A00F0
:1041E000310007F06FF80500D4E70825D2E7012574
:1041F000D0E70B25CEE70D25CCE7C046F3FF000046
:10420000F4FF000002290000D661FF1FAC61FF1F10
:104210004862FF1F332310B5040003700A220749C8
:10422000013007F0F5FA064B0F201B681A0AE372FB
:1042300022731A0C1B0E6273A37310BD0862FF1F5A
:104240003862FF1F30B5012503790400BFB02B424F
:1042500013D00B49408806F0A1FB28420DD06A46D6
:10426000084B02A81B889380FFF7D4FF6B46D880C9
:104270000022608801A903F071FC3FB030BDC04648
:10428000CE61FF1F7E41FF1F10B5024804F0E8FA1F
:1042900010BDC0464542001170B5160004AA14882E
:1042A00005AA15784A685078117800022A4A08430E
:1042B000801805284BD807F0D3F903131E29343F83
:1042C0000720022C0BD80322121BAA4200D92A0075
:1042D00022491A803000091907F09AFA002070BDAF
:1042E0000720112CFBD81222121BAA4200D92A0047
:1042F0001B491A80EEE707200E2CF0D80F22121B64
:10430000AA4200D92A0017491A80E3E70720032CA4
:10431000E5D80422121BAA4200D92A0012491A80A9
:10432000D8E70720032CDAD80422121BAA4200D9AE
:104330002A000E491A80CDE70720022CCFD803228D
:10434000121BAA4200D92A0009491A80C2E700229A
:104350000A201A80C3E7C046DCD5FFFFBEBA0011B1
:10436000F461FF1FAEBA0011A9BA0011A4BA00117E
:10437000A0BA001110B50D21024A034806F086FAD2
:1043800010BDC04694BA00119441FF1F10B5084CEF
:10439000E368002B08D18022064B52021B689B1851
:1043A0006360054B1B68236007F0AAFAA06010BD8C
:1043B0003862FF1FC8F00040CCF0004070B5184ACA
:1043C000936A916A9942FBD116498A689A421FD32F
:1043D0009A1A8B60144B0126186893B2D202D20E3F
:1043E0004343424300204C681B0A1B1912029B18CE
:1043F0000E4C0A684B60551CA3420CD8002801D013
:104400004B600A600A4A136008680A4B186070BD66
:10441000581E821ADDE7084A30009B182A00EAE796
:1044200000F000403862FF1F140AFF1F40420F00D7
:10443000C8F00040CCF00040C0BDF0FF70B51F4C8C
:1044400023793F2B01D93F2323711D4B22791A7009
:104450001878C0B207F074F918231A491A4A0B8069
:104460001A4913800B805380A379194980200B804F
:104470000C21938001334B43164D191C00018342DC
:1044800000D9011C2980D1806379002B01D101332F
:104490006371237A012B01D8022323726279237A74
:1044A0000D4853430A21584307F0C2F90B4D2860C9
:1044B000E379052B01D81023E37170BD2C62FF1F37
:1044C000480AFF1F7E42FF1FCC43FF1F7C42FF1F95
:1044D0007A42FF1F7842FF1F710200001462FF1F23
:1044E00070B520210020FEF701FF0C4C002805D1FB
:1044F0000B4B23CB23C4FFF7A1FF70BD0C22200080
:104500000849FEF7C7FE0C2802D0054B23CB23C475
:104510001C2205490548FEF7BDFEECE72C62FF1F93
:10452000DCBA0011FC0C0000D1F100008961FF1F12
:10453000F0B51D4C8022A544040088206946520134
:10454000400506F07DFF902212016A44130020000E
:1045500032C832C316C816C38023144C144FA66841
:104560009B033343A3603B6007F0BAF88823A0683D
:104570005B05C01806F02CFF002588232900802247
:10458000A0685B05C01840196944520007F088F81C
:1045900080230135FF355B019D42EED1A6603E6070
:1045A000044B9D44F0BDC046FCEFFFFF3C43FF1FA2
:1045B0009808FF1F04100000F0B5040087B0002821
:1045C00025D0684606F014FF1B4C022806D10622AF
:1045D0006946200007F03CF8002816D06946002301
:1045E00001250F262F00E25C0133100910308740AF
:1045F00038002F00324097403A0002434A610439A4
:10460000062BEFD16846FFF793FF07B0F0BD1822E5
:1046100069460A4806F014FF6A46A300D3580133DE
:1046200005D01822FF21684606F01AFFEAE7013498
:10463000062CF1D1E9E7C0466509FF1F000900110A
:10464000F0B5002704000E00150085B0BA4200D175
:104650009EE04A1C0B7801924A788978090211433E
:10466000F27812040A43317903700906114300916C
:1046700003914770232B41D8172B1DD8BB4200D183
:1046800081E0981FC2B20B2A28D9012B3ED1B84A2B
:10469000AB1E0092132B07D87378002B00D0D9E102
:1046A00000F0C8FA00F0FEFAB24B00991F78601CC7
:1046B0007A1E07F0ADF86BE0180018380B28E4D824
:1046C00006F0AEFE8900B0002C01E3FFE3FFE3FF3C
:1046D000E3FFE3FFE3FFE3FFE3FF8F010B28D4D801
:1046E00006F09EFE2F012801D3FFD3FFD3FFD3FF97
:1046F000D3FFD3FFD3FFD3FF9101B101562B64D079
:104700001FD8332B00D168E1552B44D0DB2B00D0D0
:10471000ACE1042D00D882E01027052D05D06F1FD5
:104720003A000098711D07F073F80522310020004F
:1047300007F06EF83A000099601D07F069F8053738
:1047400026E0712B00D103E1722B00D13CE1DC2B80
:10475000DCD1022D63D973784370B37883706B46D4
:104760001F88032D05D0033D3900AAB2F01CFEF7C7
:10477000CBFC39001022E01CFEF78CFDC71C002882
:1047800006DA6070D1E00C227B4907F041F80C2773
:10479000380005B0F0BD6A1E784D0C2A13D8002AE7
:1047A0000AD02800019907F033F8FFF747FE0C22E2
:1047B00028007349FEF7A8FC0C222900601C07F0B2
:1047C00027F80D27E4E70C22EBE76C4D6D4B2A0030
:1047D00043CB43C2E9E76C4E112D12D110223000B9
:1047E000019906F035FF00280BD010220199300006
:1047F00007F00EF8102265493000FEF785FCFFF740
:10480000D7FA102230006149FEF744FD020010285B
:1048100005D13100601C06F0FBFF1127B8E7FF232C
:10482000637082E0102D53D17778032F0DD1584D4E
:104830000E22B11C280006F0EBFF0E222900A01C5E
:1048400006F0E6FF67701027A2E7042FE7D1514D6D
:10485000B11C0E22280006F0DBFF29000E22A01C4E
:1048600006F0D6FF4A4D4C4E1C222900300006F0BF
:10487000EFFE002829D01C222900300006F0C8FFD6
:104880001C2230004549FEF73FFC40232A785B425A
:104890001343290028002B7000F034FA404E062202
:1048A0002900300006F0D4FE00280ED00622290090
:1048B000300006F0ADFF06223A493000FEF724FC36
:1048C0000123394A11780B43137004236370BAE74C
:1048D000022DA4D17678012E10D12F4D1C22280054
:1048E0002E49FEF7D7FC1C2806D10E222900A01C59
:1048F00006F08EFF6670A6E7FE2391E7022E8ED1AA
:104900001C2225482549FEF7C5FC1C28F4D10E229F
:104910002649A01C06F07CFF657094E7022D06D1A5
:104920007378002B03D101F085F9022730E701F0FD
:104930006FF9FAE712221E49601C06F069FF13277F
:1049400026E708221B49601C06F062FF09271FE7C3
:10495000012D35D07178F02900D960E7164D2888EF
:1049600001F09EFC154B2A885200D35A58E7C046E6
:104970002964FF1F2764FF1FE8BA00112C62FF1F84
:10498000FC0C0000DCBA00115061FF1F0DBC0000E0
:104990006D61FF1F7B61FF1F8961FF1FD1F1000067
:1049A0006509FF1FADAC00002862FF1F9761FF1F64
:1049B000F461FF1F4043FF1F8042FF1F8864FF1FF9
:1049C0003C4A3D4B1288CFE73C4B012D03D0727817
:1049D0001A704270A9E71B7822E7FFF71BFC07005B
:1049E000D6E6042D05D9364D009B2B6006F088FFD6
:1049F000A860FFF7E3FC0422039003A9601C06F003
:104A000007FF0527C4E62F4E062D15D906223000D4
:104A1000019906F01DFE00280ED0062201993000F3
:104A200006F0F6FE062228493000FEF76DFB012352
:104A3000224A11780B43137006223100601C06F0E5
:104A4000E7FE0727A4E6012D00D1E8E67078FFF71E
:104A5000B3FD6AE7013D2A000199009806F0D8FEEF
:104A60001A490098AAB2FEF74FFB1BE6DA2B00D0DA
:104A7000D5E6042D00D8D2E6082D17D9B37972797E
:104A80001B021343F27912041A43337A1B061343B1
:104A9000009A1360009B05221B68310020000393DD
:104AA00006F0B6FE0422601D03A94DE7FE236370E5
:104AB000F0E7C0468042FF1F8864FF1F2862FF1F87
:104AC0003862FF1F6509FF1FADAC0000AEDE0000BD
:104AD00070470000020010B5094B0A32094C92B22F
:104AE000DA815A8298811882207802F03FFA0422F3
:104AF000054B012120781A7006F0BAFD10BDC046A2
:104B0000CA42FF1F7264FF1F7164FF1F013870B536
:104B1000042809D806F0A4FD030927081200204B39
:104B20000221187806F0A4FD70BD1D4B08211878ED
:104B300006F0AEFE00221B4B1A74F5E7802200241B
:104B4000184B52001A82FA22DC74174B144D5B7A10
:104B5000920008215A43287806F0BAFE21002878EE
:104B600006F076FEE0E70E4B0821187806F090FE7E
:104B70000E48FFF79DF90C4B0D4A9B7993800D4A27
:104B800013800022074BDA740132FF321A820A4B7B
:104B90001B78002BC8D0094A136006F041FEC3E71A
:104BA0004862FF1F1462FF1F2C62FF1F8942FF1F14
:104BB000CC43FF1F7A42FF1F2862FF1F34F00040E2
:104BC00010B5002909D1092807D1063805F012FBD4
:104BD000024B8021187806F04BFD10BD4862FF1F84
:104BE00010B5012909D1092807D1063805F002FBC3
:104BF000024B8021187806F03BFD10BD4862FF1F74
:104C00000300F0B50A4D8E18B14202D1520080184F
:104C1000F0BD0C782F6824093C5D0F271C700C78C0
:104C200001313C402F683C5D5C700233ECE7C046CC
:104C30007442FF1F0C22124B10B51A700B23114C3B
:104C400011492370093A023B1048637006F0E0FDF9
:104C50002D2301220E490F486371FFF7D1FF012276
:104C60000D49FFF7CDFF01220C49FFF7C9FF0300F3
:104C700000200B4902001870FEF746FA10BDC0462E
:104C80004664FF1F2764FF1FBEBA00112964FF1F7F
:104C90006709FF1F2D64FF1F6609FF1F6509FF1FBE
:104CA000AEDE000070B5134C142220001249FEF74E
:104CB000F1FA431E114D132B19D8AB78002B16D0E7
:104CC000431C2B7009236B70002300190370287894
:104CD0000B4B01302900C0B2187006F079FD29781D
:104CE00022000139C9B2002005F0EEFC70BDFFF7CB
:104CF000A1FFECE72964FF1FAEDE00002764FF1F61
:104D00004664FF1FF0B54A784F790E79CD788C78DC
:104D10000B78077046708570C47002714371F0BDE6
:104D200010B5114B1A781870002A0ED000280BD13C
:104D30000E4B1A78062A07D85423D340DB0703D535
:104D40000B4B187802F012F910BD0028FCD0074B6D
:104D50001B78012B02D0033B022BF5D8044B012119
:104D6000187806F085FCEFE74A64FF1F7164FF1FA7
:104D70007264FF1FF7B5574D574A584928700920EC
:104D800005F02EFB0121032005F034FA032005F085
:104D900015FB06F00DFD032251495248FFF730FF85
:104DA0002D24030088211C70042249050130FFF7DF
:104DB00027FF302304704C4E4C4C437083702E3BC5
:104DC000062230004A49E387FEF764FA062813D02A
:104DD000300006F00DFB022809D00321300006F058
:104DE00027FC8D23F3706E3B3371193373710622E8
:104DF00030003F49FEF788F93E4B1B68FC335E6488
:104E0000FFF750FFFEF7D4FF0020FFF789FF3A4E6F
:104E100080223168394F08000197394B394F1040D3
:104E200011424FD07D3A01981A70FFF789F8387017
:104E30003A78354F01213878019B02F059F8334A0E
:104E4000334B12783878002102F052F80122314BAE
:104E5000314F1A70314B5B78552B35D1193B7B7430
:104E60002F4A304BA381E28123826282202128785D
:104E700006F016FB0120404205F072FC0120404282
:104E800005F00EFDFFF776FAFEF792FE0120404294
:104E9000FFF702F9012006F0C3FBF02001F0E4F96E
:104EA0000121287806F0E4FB287802F0BBF91E48BF
:104EB00006F04EFCFEF722FD1C4B1D4A9B689B181A
:104EC000BB60F7BD1870B3E76422737953431A00CF
:104ED0000A32C7E74862FF1FC14B0011E14B0011C6
:104EE0004043FF1FF461FF1F6509FF1FCA42FF1FF8
:104EF000ADAC00008464FF1F2C62FF1F8942FF1FBE
:104F00002664FF1FA842FF1F7264FF1F4664FF1F35
:104F10002764FF1F1864FF1F1462FF1F2862FF1F12
:104F2000CE090000C40900004A62FF1F3862FF1F5B
:104F30000000B8FCF8B50A0020230D001A40194201
:104F400000D16FE0824B1B78002B41D0FFF736FA7F
:104F5000804B814C814E99686268737A8A1ADB03B0
:104F60009A4238D36160FEF7C9FC637C002B2CD0D9
:104F7000013BDBB26374002B27D1794B5B78552B57
:104F800001D106F04DFCE37C764F002B36D000219A
:104F9000032005F02FF9F3796374BB78002B14D14B
:104FA000A27C002A02D0A374FEF73EFD3B886E4E21
:104FB000013330003B80FEF77BFF310006F0B0FB91
:104FC0000023C820E374FFF785FD237C013323749D
:104FD00020206840F8BDA37C002BC6D00023A3741A
:104FE000FEF722FD5F4A604F1388380001331380BB
:104FF000FEF75EFF390006F093FBB6E7A27C002ABD
:1050000002D0A374FEF710FD3B8801333B80564F5E
:105010003800FEF74DFF390006F082FB64237079FB
:105020005843D0E70BB2002B0ADA504B187806F041
:1050300087FC002801D006F023FC80200002C8E78E
:105040000224214206D0444B01201A74FFF768FE67
:105050002000BEE780246400214202D000F05CFD05
:10506000F6E70824214204D0FFF7A8F9FEF746FC32
:10507000EEE710230E001E4019420FD0FEF7D4FCBD
:10508000334B1B78002B07D1FEF7A6FD334B1B6873
:10509000DB0701D5FFF7F8F810209AE70124214239
:1050A00009D0334800F0B4F806F052FC3100032078
:1050B00005F0A0F8CCE70B0641D5092004F066FF07
:1050C000284E071E2CD0737A234205D01A000123E4
:1050D0001343737280207CE71F4B717ADA681F4894
:1050E0000132DA600122114371721949B2700978F4
:1050F00000291CD03188DA7401313180C2791A4C10
:105100005A74144A1B499268200052189A60FEF79C
:10511000CFFE210006F004FBC820FFF7DBFCD9E737
:1051200000F088FD737AB770A3437372D2E7036807
:105130001342CFD0FFF742F9FFF7A6F8CAE70424DD
:1051400008002040214200D144E7FEF7C1FF7FE77D
:105150004A64FF1F3862FF1F1462FF1F2C62FF1F8B
:105160002862FF1F0862FF1F8942FF1F4862FF1F5E
:105170006C42FF1F000082FCF0B51B4B1B4F1B88CD
:105180003A8804001A4E1B4D85B09A420DD83288D9
:105190009A420AD3184B1A882B889A4205D1174A8B
:1051A000174B12881B889A421BD0052001F0B2F8D9
:1051B0003B8802AA13803388019053802B88114DBD
:1051C00093800F4B02A91B88D3800F4B2A78188835
:1051D00002F0CEFD0D4B08212878019A1C7006F0D4
:1051E00067FA05B0F0BDC0461664FF1F7E42FF1F80
:1051F0007C42FF1F7A42FF1F1464FF1F1264FF1FCF
:105200007842FF1F7264FF1F8042FF1F1064FF1F60
:1052100013B50C4B1C78002C11D1002801D00A4B7F
:1052200018600A4A0A4B11780A4A10780A4A019211
:105230000A4A0092002205F03FF9200016BD112411
:10524000FBE7C0467164FF1F0C64FF1F7064FF1F03
:105250006064FF1F7264FF1F4C64FF1F5064FF1FD8
:1052600010B5064B12201B78052B06D1044B1322D8
:105270001988044B187801F029FA10BD7164FF1FDA
:105280008042FF1F7264FF1F10B500240122114BE2
:1052900052421870104B1C70104B1A8001F0C2FF64
:1052A00004220F4B21001A700E480C3206F030F920
:1052B000102221000C4806F02BF907220B4B1C6032
:1052C0000B4B1C700B4B1C700B4B1A700B4B1C7058
:1052D00010BDC0467264FF1F7164FF1F8042FF1F34
:1052E0007064FF1F6064FF1F5064FF1F4C64FF1F4A
:1052F0002664FF1F2564FF1F8242FF1F2464FF1FD7
:10530000F8B5174C0600257806A814240078052D5A
:1053100023D1B41F134FA5B21824BD421DD88D1F31
:10532000ADB2BD4219D8FA256D00AA4215D21D00B2
:105330000D4F0A3DADB2BD420FD80C4C26800C4C2F
:1053400021800C4900240A800B4A1380FFF714FFC8
:105350000A4B0421187806F09BFA2000F8BDC046DD
:105360007164FF1F790C0000750C00007E42FF1F66
:105370007C42FF1F7A42FF1F7842FF1F7264FF1FAB
:10538000F0B50BB20D0089B0002B00DB70E1A44E2C
:10539000307806F0D5FA041E50D00378A22B00D145
:1053A00022E1D02B1AD0912B45D143780E2B42D13C
:1053B0009C4B82889A423ED19B4A83681278052A88
:1053C00039D1032018567F2835D0984B1B68002B05
:1053D00031D05B68002B2ED098472CE080780728CE
:1053E00029D806F03DF90428183F3F74A8D86378FF
:1053F000002B0CD101218C4B19708D4B1A78002A8F
:105400005BD08C4B307801F073FD002855D007221B
:10541000854B1A7051E061780029F8D1E378002BB0
:1054200011D0854A854B1278307801F061FD6070AB
:105430006378002BEBD1200006F022FA80200002D6
:10544000684009B0F0BD784B1B78022BF3D00121E6
:10545000307805F0DDFF0028EAD10121307806F030
:1054600007F9E5E76378002BD1D16F4F032807D107
:105470003B78052B02D101333B701EE00223FBE792
:105480006F4B1A886F4B0293002A0BD01B78002BAE
:1054900003D00121307806F00BF93B78062B04D1BC
:1054A000013BE9E7029B1A70F7E7042B41D1012188
:1054B000029B3078197006F0DBF85C4B1B68002B00
:1054C000B9D01B68002BB6D0574A107884E76378B0
:1054D000554F002B27D10622211D5B4806F098F975
:1054E00062895A4B5A491A80A2895A4B1A80E38919
:1054F0000B800521397058490A80584A1380228A46
:10550000574B1A80574B1B78012B09D11F2000F0F5
:1055100001FFFA22920042430421307806F0C8F8D5
:105520000022484B75E7312B00D070E70022454B35
:105530001A700323A0E706220021434805F0E8FF84
:105540000023454A04211380444A30781380444A9A
:10555000138006F09DF90821307806F099F9A379B7
:10556000083B5A425341304A03331370304B1B7887
:10557000002B06D0334B30781A78002A06D001F081
:10558000F5FC0122314B52421A8096E70121197035
:1055900006F06EF8F5E70821307806F079F96378BF
:1055A000002B00D047E72C4B2D4F0293E388029A43
:1055B00004211380294B307803932389039A1380A5
:1055C00063893B8005F024FF002800D033E7264B99
:1055D0001B68002B00D12EE7039902983A880988AE
:1055E00000881B68984726E74379132B00D022E7F1
:1055F0000389012B0AD11D4B1B78022B06D10821F0
:10560000307806F045F9FFF72BFE14E7052000F08F
:1056100081FE08210200307806F04AF80BE7C04608
:105620007264FF1F051400007164FF1F0C64FF1FEC
:10563000A842FF1F8942FF1F4664FF1F2764FF1F08
:105640004864FF1F4A64FF1F1964FF1F8042FF1F49
:105650002064FF1F2264FF1F1664FF1F1464FF1FD6
:105660001264FF1F1864FF1F0864FF1F1064FF1FF0
:105670008020C001014200D0E2E6CB0731D5324B99
:105680001B78002B1DD0314E05AC3378052B1AD179
:10569000023B23702E4B21001B7823722D4B1B786D
:1056A00063722D4B187801F0C7FB002809D0072042
:1056B0002A4B30701B68002B03D01B68002B00D0D6
:1056C00098470120BCE60E20254B06221B78254971
:1056D0002370254B1B78637002ABC01806F098F856
:1056E000D8E7022308001840194209D0174B1B784D
:1056F000052B03D11D4B188806F042F802209FE6C7
:105700000424214203D0FFF737FD200098E6082348
:1057100008001840194200D193E6154B1C78012C63
:1057200003D0022C0DD008208AE6124B124A1349EE
:1057300013481B881288098800880094FFF7E0FD51
:10574000F1E7FFF78DFDEEE74A64FF1F7164FF1F6D
:105750008242FF1F2464FF1F7264FF1F0C64FF1F3F
:105760002664FF1F8342FF1F2564FF1F8042FF1F27
:105770001064FF1F7842FF1F7A42FF1F7C42FF1F09
:105780007E42FF1F0200F0B501270A480A4E511859
:105790008B1A002B00DCF0BD082415784308684004
:1057A00038404000805B013C58406D08002CF5D12A
:1057B0000132EDE7FFFF000006BB0011F0B5002548
:1057C0000F269D4200DBF0BD4C5D0709444034408C
:1057D000A400A05801357840F3E70000F0B589B087
:1057E0006A460D000B000F27110010351C7801339D
:1057F000260024093E40167054700232AB42F5D1A7
:105800002023024AFFF7DAFF09B0F0BD0CBB0011FC
:10581000F0B54E780B7889B036020C001700019075
:105820001E43012A61D9954B9E4200D877E001338F
:105830009E421CD1062A17D1CA788B7812021A43CD
:105840000B791B0413434A7912061A438C4B5A6195
:1058500000221A705A808B4A5A608B4A9A608B4A8F
:10586000DA60002009B0F0BD88225205EEE7884BCF
:105870009E423CD182498B78002B00D0F6E00C2A66
:1058800031D10F22A3789343E27812021343227995
:10589000120413436279120613434B60E279A07934
:1058A00012020243207A00041043627A1206024375
:1058B000CA60E27AA07A1202024376484A818342A1
:1058C00008D804236E49142201980B7005F0A0FF3C
:1058D0001420C7E71201D21889235B059A42F0D839
:1058E00001238B70BDE7022AFAD00523EAE76A4A52
:1058F00001239642E6D1FFF7B3FC052F0CD9E378DC
:10590000A2781B021343227912041A4363791B06FF
:105910001343624A0393136005F082FFA1E7584DD9
:105920002B78002B9DD1AB78002B00D1A0E02B89E8
:1059300001339BB20093B34200D091E0132AD4D933
:10594000CF7C8B7C3F02122120001F43FFF71AFF00
:10595000874200D08EE0002E3DD1E378A2781B0272
:1059600013432279E96812041A4363791B0613432F
:1059700003930A228B4212D1FF23A370E370237199
:1059800063716B89002B09D1E37B227C1B0212041B
:105990001343A27B13431B0901336B8100226B89E4
:1059A000002B8ED0002A67D1686837013818000BA9
:1059B0006B6900030390984205D9686105F008FD02
:1059C000EB780133EB7068681022A11C381805F0E1
:1059D00067FE2E8145E76F89009A7B1E9BB293423A
:1059E0003AD1E278A37812021A43237905A81B045E
:1059F000134362796C6812061A43EB6800920392B3
:105A0000211D0C22049305F003FF0120260004A9A8
:105A100040421036FFF7E2FE013F012F17D1009AF6
:105A20000B232861824200D04CE704221C4920004D
:105A300005F036FE042203A9686805F001FDE96857
:105A4000039AFF23914200D13CE7F73B3AE731004C
:105A5000FFF7C4FE1036DFE70923B742A4D831E7C9
:105A6000009BB34200D9FCE607232BE7022329E77A
:105A7000032327E7062325E70A2323E7FFFE000089
:105A8000AC42FF1F00000111FFFF000050485936D3
:105A900001FF0000FFFF001102FF000034F0004092
:105AA000B842FF1F0121174BF0B51A68164C8A4304
:105AB0001A601A688606B60F2240340322431A6021
:105AC0001A68124C870922401A604022BA403241BB
:105AD0000F26304088400E4C12042568ADB22A4390
:105AE000226022680B4D120C405B120402432260BC
:105AF00080221868520202431A601A681143196022
:105B0000F0BDC04604E00040FF8FFFFFFFFFFEFF37
:105B100008E000404CBB0011F7B5364B364C019302
:105B20002388019A5B009D5C344FFF2D2DD103210A
:105B3000052004F04BFA0021052004F037FA01217A
:105B40002F4B12201A688A431A601A680F318A4351
:105B50001A6005F0B5FE122005F0CAFE00233B7066
:105B60002388019A5B00D318372280215B78490093
:105B70005A43244B187805F09BFD238801339BB2D0
:105B8000732B00D900232380F7BD3E78002E2DD142
:105B900032003100122005F05BFC122005F010FEEF
:105BA000122005F035FD28001025FFF77BFF164B6E
:105BB00016491A6805200A401A601A682A431A60B2
:105BC0008022196812060A431A60310004F0FEF9B7
:105BD0000A21052004F044FB0121094B1A680A43FD
:105BE0001A601A6815431D603970B9E72800FFF77D
:105BF00059FFB5E76CBB00117464FF1F7664FF1F8B
:105C000000E000404862FF1F04E00040FFFEFFFF8D
:105C1000802110B5054B4900187805F039FE0022A7
:105C2000034B1A80FFF778FF10BDC0464862FF1F84
:105C30007464FF1F01210E4B10B51A6812208A43AD
:105C40001A601A680F318A431A6005F051FE12205B
:105C500005F036FE0022074B032105201A7004F0E0
:105C6000B5F98021044B4900187805F011FE10BDEC
:105C700000E000407664FF1F4862FF1F10B5034C30
:105C80000B000122210000F06BFA10BD3D5E0011F7
:105C90000B8870B506000D000224162B11D92B00BD
:105CA0000322094900F05CFA041E0AD1074B2A8836
:105CB0001B88191C934200D9111C300089B200F0D6
:105CC000EFFA200070BDC046695E00118A64FF1FB4
:105CD00010B54A780400013A0B000220012A07D8C7
:105CE0000A78002A04D005222000024900F038FA80
:105CF00010BDC046975E00110A7810B50B00040075
:105D00000220002A04D007222000024900F028FACD
:105D100010BDC046435F00110A7810B50B000400A7
:105D20000220002A04D009222000024900F018FABB
:105D300010BDC046A95F001110B5034C0B000B222B
:105D4000210000F00DFA10BDD95F001110B5034C11
:105D50000B000D22210000F003FA10BD4B60001172
:105D600010B5034C0B000F22210000F0F9F910BD13
:105D7000A56000110A7810B50B0004000220002A6B
:105D800004D011222000024900F0EAF910BDC046FB
:105D9000B5600011002310B51322190000F0E0F9DE
:105DA00010BD000010B5034C0B001722210000F0BD
:105DB000D7F910BD07610011002310B51922190091
:105DC00000F0CEF910BD000010B5034C0B001B22F3
:105DD000210000F0C5F910BD41610011F7B58489BB
:105DE0000D0006000121002C22D000238268D3562A
:105DF0001778002B1EDA0C2C1AD90C3CA4B21319FC
:105E000040880093230002F086FE431E9841013033
:105E10007B06DB0F6B703F23013C1F40A4B2287050
:105E2000AF70AC80002C07D0B3680133AB600021A9
:105E30000800FEBD0020EBE7AC60F8E70B780370CC
:105E40004B8843704B881B0A83700B79C370042006
:105E500070470420022B06D10020537811781B02D2
:105E6000009A0B43138070470B8803700B881B0A42
:105E70004370022070470420009983420AD153786E
:105E800010781B0203430B80D37890781B020343E6
:105E900000204B807047F8B50D004B78012400219D
:105EA000461C03702B788B4201D82000F8BD6B781C
:105EB000B01C4F1C012B10D1890069184B8802229D
:105EC00033704B88B9001B0A7370691805F0F8FA33
:105ED00004360434A4B2F9B2E4E7122359436B1830
:105EE0005A88043132705B8810221B0A737069185B
:105EF00005F0E6FA12361234ECE770B5049D140092
:105F00001E00052B01D8042070BD637812781B0297
:105F100013432B80E378A2781B02134302226B8089
:105F20002A71211D681D063E05F0CAFAB2B22A8107
:105F3000E92AE8D82800A11D0A3005F0C1FA00209E
:105F4000E2E7002310B50A789A4201D8900010BD0C
:105F50009A008A185488013304705488DBB2240AEA
:105F60004470948884709288120AC2700430EAE700
:105F700010B51100029C062B04D004201022142B13
:105F800001D010BD022222714B7808781B02034316
:105F90002380CB7888781B02034363800431601D23
:105FA00005F08EFA0020ECE710B50C788B78043100
:105FB0005C43E4B203702200013005F081FA601CFA
:105FC00010BD0420022B06D10020537811781B024B
:105FD000009A0B431380704710B50C000A880231F9
:105FE00005F06EFA208810BD70B504000D0004980D
:105FF0001100012B01D8042070BD167852781202CE
:10600000324302800200F13255701470E125002CF9
:1060100000D10C35023B9AB24280AA42EBD8023141
:10602000043005F04DFA0020E6E704200099834291
:106030000AD1537810781B0203430B80D3789078F1
:106040001B02034300204B80704710B50C000A88E8
:10605000023105F035FA208810BD000070B501212D
:106060001E000420049C0E400B4218D1CB40DDB230
:106070008D4214D90A49DBB2098899420FD3230013
:10608000EE331D703300580011184978165C090270
:10609000314301332152D9B28D42F4D8002070BD72
:1060A000C442FF1F10B50C000A88023105F008FA3F
:1060B000208810BD10B50C788B7804315C43E4B2B5
:1060C00003702200013005F0FBF9601C10BD10B513
:1060D00011000298032B01D8042010BD14785278C7
:1060E000043B120222430280CA788C7812022243B7
:1060F00042809AB28280EB2AEED80431063005F055
:10610000DFF90020E9E710B50C000B8803700B885D
:106110001B0A43704B8883704B881B0AC3708A88A4
:106120000430063105F0CCF9A088043080B210BDEF
:106130000420012B03D100201378009A13707047BC
:1061400010B50C000B8803700B881B0A43704A883B
:106150000230043105F0B4F96088023080B210BD1D
:10616000F0B589B003931E4B029242000700D05A4B
:10617000019102F020F81325061E2DD0029B012468
:106180000370019B002B04D0001903999847001954
:1061900084B26B461B7A5BB2002B0FDA10213800F9
:1061A00002F01CFB1925002813D130003219E1B28E
:1061B00002F066FC051E0CD10C34A4B2042304AA20
:1061C000380005A993800696948101F0AFFD051E65
:1061D00002D0300005F094F9280009B0F0BDC046A7
:1061E0008864FF1F70B505000C0000280CD000204B
:1061F000814209D010222000044905F061F90120F4
:106200002B7823736B78637370BDC04654BC001148
:10621000F0B506000D0017001C0085B002291BD048
:106220000020102907D1022B07D0102B03D115E035
:106230000020102C08D005B0F0BD69463800FFF7EB
:10624000D1FF2A0069460BE069463000FFF7CAFF1C
:1062500022006946380004E0022BE9D12A00390007
:10626000300005F0C5F9E6E7031CF02800D9F0235B
:10627000032008499AB2013A0B80D317034006491C
:106280009B189B100B80D30F04499B185B100B804D
:106290007047C046C842FF1FC642FF1FC442FF1FCF
:1062A000034B1B888B4202D3024B4000C152704704
:1062B000C842FF1F8864FF1F014B4000185A7047F7
:1062C0008864FF1F1722014B1A8070478864FF1FE4
:1062D00070B505000E2005F003FB041E13D0D0237B
:1062E000037000230622837007494570033005F0D0
:1062F000E7F8064B2100DA8A62811B7E2373044B88
:10630000187805F0CDFA70BDA464FF1F9464FF1FD8
:106310001843FF1F262803D8024B4000C05A70477D
:106320000148FCE7CA42FF1FFFFF000070B50600EE
:106330000C00094D1C220021280005F0E9F8074B4C
:106340001E70074B1C7005F0EBF80123002801D0EC
:10635000002312202B7070BD9464FF1F1843FF1F91
:10636000B564FF1F70B505000D4C0800E260A16028
:1063700010220021656005F023FB012803D11021C4
:10638000A06802F058FD10220021280005F018FB3B
:10639000012803D11021606802F04DFD70BDC04698
:1063A0009464FF1F70B5041E05D1002903D0062296
:1063B0000D4805F085F80D4B1D78012D11D1002CED
:1063C00005D102221A7005F0EBFA280070BD0022F8
:1063D0001A70074B1B78FF2BF7D02000FFF778FFD0
:1063E000F3E70025F1E7C046A464FF1F9464FF1F94
:1063F0001843FF1F030010B5002801D1002010BD75
:1064000000780B4A002803D15988D1821B79137672
:106410001378022BF2D10023984200D1033313707A
:10642000044B1B78FF2B01D0FFF752FF0120E6E75A
:106430009464FF1F1843FF1F002911D000280CD0BF
:106440004B79012803D140225242134303E03F22FB
:106450001340032802D001204B7170474022F4E71B
:106460000800FAE770B5094D0100287800280BD024
:10647000074C0622200005F023F821002878FFF7BA
:10648000DBFF200004F0FCFF70BDC046B464FF1FBA
:106490008E64FF1F00290AD0012808D13F224B79C2
:1064A0009343C02B03D0403B5A425341981C704742
:1064B00070B5174D06002B78FF2B15D00A2005F07C
:1064C0000FFA041E10D0D0230370C83B8370114B09
:1064D00011491B784670C3700622043004F0F0FFA7
:1064E0002100287805F0DCF90C4B1B78012B0DD12D
:1064F0000B4B1B68002B03D09B68002B00D09847E8
:10650000084B04211878084A05F0E2F970BDC0462E
:106510001843FF1FB464FF1F8E64FF1FB064FF1F8A
:10652000DC64FF1FE064FF1F60EA0000014B986815
:106530007047C0469464FF1F014BDB6818687047C2
:106540009464FF1F074B10B5DA68136801331360BA
:10655000054B1878FF2803D08021C90105F088F881
:1065600010BDC0469464FF1F1843FF1FF7B50E000F
:1065700002F0C8F8051E1CD00E4B06621F78002FD3
:1065800000D10778AB791020019305F0A9F9041E1A
:106590000FD0D0230380C73B8370019BE91DC370DC
:1065A0000622043004F08CFF21003800E66005F07C
:1065B00077F9F7BD1643FF1F014B18787047C046A7
:1065C000B464FF1F054B002805D1054B1A78054B15
:1065D000002A00D1014B18007047C046A464FF1F79
:1065E000B464FF1F8E64FF1F014B58687047C0469C
:1065F0009464FF1F024B1868431E9841C0B2704755
:10660000B864FF1F421E03000120152A03D9FF3B77
:106610005A425341D8B27047F0B51C0000230E0017
:1066200085B0039002920B70029A934201D300202E
:1066300019E0E55C5A1CD2B2002DF8D0029851192D
:106640008142F4DC0233DFB2A35C18000193FFF750
:10665000D9FF002807D0013D019A0399EBB23370AE
:106660008A4202D1E01905B0F0BDDB19DBB2DBE7ED
:1066700010B50C0002F09EF803001220002B03D08E
:106680002100588804F0ACFF10BD000070B50E4D1D
:1066900084006359002B15D0186A002801D004F03B
:1066A000AFFE2B59586A002801D004F0A9FE2B59DF
:1066B000986A002801D004F0A3FE285904F0A0FE37
:1066C00000232B5170BDC046C464FF1F1C4B70B526
:1066D00004000E00150099420AD11A4B1B68002BCA
:1066E00001D1122070BD1B68002BFAD09847F9E742
:1066F000154B994215D1134B1B68002B0AD01B6810
:10670000002B07D09847002804D1104B1C70104B69
:106710001D70E7E729002000FFF7AAFF0028E1D15C
:10672000F3E7080001F0EEFF0028DAD00378032039
:10673000A342D7D12900300004F052FFD2E7C0466F
:10674000FEFF0000C064FF1FFFFF0000BD64FF1FCD
:10675000BC64FF1FF7B50400808801F0D3FF00255B
:10676000A84203D00578A08802F008F81C4E3378C0
:10677000002B1FD0AB421DD11A4B28001978FFF710
:1067800077FF002818D000233370A3790820A7785A
:10679000A688019305F0A4F8011E0DD0D023037044
:1067A000CA3B8370019B477086808371280005F087
:1067B00077F801E0002DE8D1A0880B4B8200D35878
:1067C000002B01D0FFF762FF1721A088FFF768FDBB
:1067D000A08801F027FDA08801F0FEFDF7BDC046AE
:1067E000BD64FF1FBC64FF1FC464FF1FF0B587B00A
:1067F0001D000CAB1B88070001930DAB1B881420F8
:1068000002930EAB1B88160003930FAB1B880091FD
:10681000049310AB1B88059305F062F8041E1AD090
:10682000D0230370CB3B47708370C67006222900CB
:106830000430002D11D004F043FE019B2100638140
:10684000029B0098A381039BE381049B2382059B09
:10685000A37405F025F807B0F0BD04F059FEECE78D
:10686000F7B5009308AB1B8807000C200D0016003D
:10687000019305F035F8041E13D0280001F042FF03
:1068800000280FD00078D0232370C93BA370009B51
:1068900021002381019B6770A580E680638104F05D
:1068A000FFFFF7BD014B1878EDE7C0461843FF1F07
:1068B00013B5040064890389C2888188C078009474
:1068C000FFF7CEFF13BD000010B5044C2068002870
:1068D00003D004F095FD0023236010BDC864FF1FA2
:1068E000A122F0B5818892004A43384B384F1B688B
:1068F00004009B189D2292009B18827989B01A602F
:106900003B68002B5FD01D78324B1B68002B04D0F6
:106910005B68002B01D00020984726000836310024
:10692000E079FFF7B7FD237DE0710200E078049382
:10693000638A29000393238A0293E3890193A3883E
:1069400000933300FFF752FFE378002B0BD1E2896D
:10695000A379A18802920196E2792800009201228F
:1069600001F0DAFEE0703B68002B20D0FFF7ACFFAF
:10697000194D287800281AD0184B1978FFF778FE9F
:10698000002814D02B78E67808200793A78804F015
:10699000A7FF011E09D0D0230370CA3B4670837045
:1069A00087808671079804F07BFF00232B701721E6
:1069B000A088FFF775FCA08801F034FCA08801F0E6
:1069C0000BFD09B0F0BD064B9DE7C0463409FF1F23
:1069D000C864FF1FDC64FF1FBD64FF1FBC64FF1F92
:1069E0001843FF1FF8B5070008000E0001F08AFEEB
:1069F000041E18D02620FFF78DFC051E00D1257837
:106A0000062004F06DFF041E0DD00021062204F0C4
:106A10007FFDD0232370C23B21006770A370A68046
:106A2000E8B204F03DFFF8BDF0B585B001930AABC4
:106A30001B78070002930BAB1B7808000D00009237
:106A4000039301F05FFE061E22D0102004F048FFE1
:106A5000041E1DD01022002104F05AFD2620FFF74D
:106A600059FC002800D13078D0232370C13BA3709B
:106A7000009B21002372019B67706372029BA580BB
:106A8000A372039BC0B2E3720C9BE36004F008FFA7
:106A900005B0F0BDF7B50D00019001F033FE071E03
:106AA00020D00E2004F01CFF041E1BD02620FFF770
:106AB00031FC061E00D13E78D0232380C53B062240
:106AC000A370F91DE01C04F0FBFC019B2A0063810C
:106AD0000123DD401A401D40210022736573F0B28E
:106AE00004F0DEFEF7BD0000F0B585B002901000A6
:106AF0000D0017000A9E039301F004FE041E31D01E
:106B0000029B002B2ED1039B02795B0724D5122315
:106B100013430422002E08D10B99002905D10C99AA
:106B2000002902D10D9900291AD01A430D9B227118
:106B3000002B00D0C9E0002E00D1CFE0002D00D006
:106B4000CCE0606A002801D004F05AFC1C2130001F
:106B500004F016FF606205E002239A430E33D7E784
:106B600093432371654BBA00D458002C00D1AAE09E
:106B7000002E10D0236A002B03D11C2004F078FED5
:106B800020625E4BBA00D358186A002803D01C223A
:106B9000310004F095FC0C9B002B12D0574CBB002D
:106BA0001D596B6A002B03D1162004F061FE686248
:106BB000BB00E358586A002803D016220C9904F051
:106BC0007FFC0D9B002B11D04C4DBC006659B36A65
:106BD000002B03D1142004F04BFEB0622B59986AAD
:106BE000002803D014220D9904F06AFC380001F04B
:106BF00089FD051E67D0414BBA00D358002B62D0E7
:106C00001A6A3420002A00D11C389A6A002A01D05E
:106C1000143080B20B9A002A01D01C3080B25B6A1B
:106C2000002B01D0163080B204F05AFE041E4AD068
:106C30001822002104F06CFC2620FFF76BFB01906A
:106C4000002801D12B780193D0232370029B2000D0
:106C500063700A23294EA370039BBD00A371AB5937
:106C6000A780196A1830002905D01C22A06004F002
:106C700027FC200034307359996A002907D003009B
:106C800014221433E060029304F01AFC02980B9B68
:106C9000002B08D003001C221C330B9920610293A7
:106CA00004F00EFC02987359596A002903D0162289
:106CB000606104F005FC6B462100187904F0F0FDDA
:106CC0003800FFF7E3FC05B0F0BD10220D9B0D99D5
:106CD0001B69A018236204F0F3FB2CE70B9B002B2D
:106CE00000D13FE7012D00D03CE7606A002801D0C9
:106CF00004F086FB1C210B982AE7C046C464FF1FE2
:106D000010B5044C2068002803D004F079FB002360
:106D1000236010BDB864FF1F0B4B07B51A68002A2B
:106D200001D100200EBD6946531C012012780731A5
:106D3000FFF772FC0028F4D00278012310001840FD
:106D40001A42EED0EEE7C046D464FF1FF0B51F4FE5
:106D500001203B6887B0002B25D09B78059300F07D
:106D6000B3FB002821D00A20FFF7D4FA04000B203F
:106D7000FFF7D0FA164B05001E78731E9E413B6844
:106D8000F6B2191DD878FFF757FB3B682900DA7A6D
:106D9000043303929A790193029200903300200009
:106DA000059A04F085FD07B0F0BDFFF7B5FF002898
:106DB00005D00620FFF7AEFA04000720D8E7082028
:106DC000FFF7A8FA04000920D2E7C046B864FF1F05
:106DD000B464FF1F70B50A4E040033780D00FF2B1A
:106DE0000DD0042004F07CFD011E08D0D0230370D8
:106DF000CE3B45708370C470307804F051FD70BD97
:106E00002843FF1F70B5040006200D0004F068FD44
:106E1000011E0AD0D0230370CD3B8370054B447014
:106E20001B688580187804F03BFD002C01D0FFF72B
:106E300067FF70BDB864FF1FF8B5264F06003B68BA
:106E40000D001124002B05D10522234B1B78134282
:106E500002D112242000F8BD204A10241268002A12
:106E6000F8D01278002AF5D0DB0719D52B789A1EB6
:106E7000012A1AD80C2004F0FBFC132438600028E7
:106E8000E8D000230A22437029000670023004F083
:106E900017FBFFF75BFF041E0AD0FFF731FFD9E7AE
:106EA00000F012FB0028E1D1E4E7002BE2D0D0E7AC
:106EB0000B4B1B78032BCDD11D20FFF72BFA094B71
:106EC00018800028C6D0084B04211878074A04F01F
:106ED000FFFCBFE7B864FF1FB564FF1FD464FF1F4A
:106EE000B464FF1FB264FF1FE064FF1F60EA00008C
:106EF000F7B50193194B14001A78052306000F000B
:106F000012201A4221D0012920D1154B1D68002DD5
:106F10001BD002201F2C18D8002C02D0019B002B64
:106F200013D0104B1F221E706E1C0021300004F085
:106F3000EFFA01992200300004F0C2FA310020007B
:106F40002C70002F06D004F013FDFEBD064B12205E
:106F50001D68DCE704F03CFCF7E7C046B564FF1FA2
:106F6000D464FF1F2843FF1FD064FF1FF8B50F4EE6
:106F700012243368002B17D01B780F3C834213D1A7
:106F800000250B4F0221387804F082FC094B0421C4
:106F900038781D8004F07CFC074B28001D80336886
:106FA0005C7004F085FA04002000F8BDB864FF1F8F
:106FB000E064FF1FCC64FF1FB264FF1F70B501289F
:106FC00023D11B4C2388002B03D01A4A1578002D9F
:106FD00007D0194B1B68002B02D01878FFF7C6FFAB
:106FE00070BD3B2B02D93C3B2380F9E7134E0221B5
:106FF000307804F04DFCFA222388920002215A4393
:10700000307804F055FB2580EAE70B4B1B68002B1A
:10701000E6D00B4B1B785B07E2D5084B02211878B2
:1070200004F036FC0022024B1A80FFF769FED7E716
:10703000CC64FF1FB064FF1FB864FF1FE064FF1F34
:10704000B564FF1FF8B51E4D2868002803D004F072
:10705000D7F900232B601B4E3068002803D004F0C2
:10706000CFF900233360184F05243B7818002040E7
:10707000234221D0154800F02BFA3B78234213D04D
:10708000202004F0F5FB2860002813D020220021E6
:1070900004F03EFA202004F0EBFB041E306005D023
:1070A0002022002104F034FA002004E0286804F0D3
:1070B000A7F92C601320F8BD00F00AFAF4E7C046E7
:1070C000D464FF1FD064FF1FB564FF1F1C43FF1F64
:1070D00010B50A4C23681A1E0ED0002808D10130C2
:1070E000587004F0E5F9002805D02368002B02D081
:1070F0000021FFF787FE0122100010BDB864FF1FBA
:10710000F7B5274E050033680191181E21D05C7831
:10711000244F012C30D1FFF7FFFD002825D020009F
:10712000FFF7F8F80400412814D91F4B0221187802
:107130001E4A04F0CDFB1E4B3C3C1C8002223368EF
:107140005A703B78002B14D128000199FFF75AFEA2
:107150000120FEBDFA2292004243002AEED0124BDB
:107160000221187804F0A4FAE8E7FFF7D3F8020048
:10717000F3E700233B70EBE73B78002BE8D10320DB
:1071800004F0AEFB011E08D0D0230370CC3B457049
:1071900083703368187804F083FBFFF7B1FDD7E7FD
:1071A000B864FF1FB064FF1FE064FF1F60EA0000C7
:1071B000CC64FF1F10B51749838802008B4220D092
:1071C00011D815498B4217D0144900205B1899B289
:1071D000012907D8926811785A425341D8B2FFF773
:1071E000F9FD012010BD0E4A00209B1807229BB21A
:1071F0009A424041C0B2F5E783681878FFF768FF0C
:10720000F0E7836899785A78090218781143FFF7F4
:1072100077FFE7E70A20000006200000F8DFFFFF05
:10722000AFDFFFFF014B18707047C0462943FF1FB7
:1072300010B5064C207001F041FA207804F0C0F837
:107240000521207800F062FD10BDC046E064FF1FFC
:107250000BB273B50D00002B00DBC4E0884B18782F
:1072600004F06EFB041E0ED00378912B0FD0A22BDE
:1072700000D1A1E0834B1878FF2852D0210004F000
:107280000FFB00284DD180200002684076BD437876
:107290000F2B76D013D8052B70D00E2BEAD1808817
:1072A000794B98422BD8794B98421BD8784B98420F
:1072B000E0D1A3681878591CFFF774F838E03E2B2A
:1072C000D8D18378032B74D06CD8012B6ED0022BCD
:1072D000D0D1704B1B68002B23D05B68002B20D0D3
:1072E00098471EE06C4BC0180C28C3D804F058FA1D
:1072F0001DC2C2150BC20B0B0B3223C23C00674BE5
:10730000C0180728B6D8664B1B68002B09D01B682D
:10731000002B06D0200098470AE0A3681878FFF7F2
:10732000C7F8200004F0ACFAADE7A068FFF762F8F8
:1073300000289FD0F5E7A3681B78002BF1D0554BB0
:107340001B68002BEDD01B68002BEAD021005548AC
:107350009847EDE74F4B1B68002BE2D01B68002BD2
:10736000DFD021005048F3E7504B1B68002BD8D0EA
:107370005B68002BD5D021004348E9E7FFF7EAF925
:10738000CFE780884A4B984203D04A4B984200D0BE
:1073900070E7464B1B68002BC3D05B68002BC0D046
:1073A0002100D5E7153B012BBBD963E7FFF798FA1E
:1073B000B7E7FFF77DFAB4E73F4B1B78042B07D103
:1073C00000236A4613800179408800F0C5FCA8E7D5
:1073D000364B1B68002BA4D05B68002BA1D00100AA
:1073E000364898479DE7012421420AD0294B1B6863
:1073F000002B04D05B68002B01D0002098470120AF
:1074000043E78B070AD5264B1B68002B04D05B682B
:10741000002B01D020009847022036E704212800E5
:1074200008400D4200D131E7254E3388002B21D092
:10743000013B9BB23380002B1AD1FFF7DBF8002809
:107440000AD0204B1C70164B1B68002B04D05B68C5
:10745000002B01D020009847FFF7C6F8694601F0DD
:1074600001FD6846FEF7FEFF1D20FEF753FF30804A
:1074700004200AE7024B187804F00AFAF8E7C0463D
:10748000E064FF1F2943FF1F0E20000001200000C1
:1074900009100000D864FF1FFEDFFFFFAFDFFFFF12
:1074A000DC64FF1F0C2000000B200000C064FF1FE5
:1074B0000D20000013200000B564FF1FFFFF000037
:1074C000B264FF1FB064FF1F10B501F09BF910BD3F
:1074D000014B18607047C046DC64FF1F0B8800201A
:1074E000162B01D817230420014A13807047C04689
:1074F0008A64FF1F00207047074A030011888142F9
:1075000007D091880020994202D1013080001018E4
:1075100070470020FAE7C046E864FF1FF0B58F7897
:1075200006000D00C5B01E2F15D1FFF7E5FF051EA3
:1075300003D10024200045B0F0BD00223B00310003
:10754000C078009200F0B2FB0400A81C00F0D2FB4F
:10755000FF23EB70EEE7264B062403931B78FF2BEB
:10756000E8D0182FE6D87B08224A013BDB000292C4
:107570009A589446002ADDD0029AD3185B68002BF3
:10758000D8D00878002802D14B78012B02D10624EC
:10759000122FCFD107AFAB88697800976446AA68ED
:1075A000A047041EC6D1AB78029A5B08013BDB0002
:1075B000D318390030005B689847041E0BD1AB78B4
:1075C000042BB6D0039A310010782200009700F007
:1075D0006DFB0400AEE76A78002AABD1AA7805A952
:1075E0003B88087130000A704B80FEF747FBA0E72C
:1075F0002C43FF1F64BC00111D4B37B5050098429A
:107600000BD000290AD1FFF777FF002805D11948D0
:10761000FFF772FF002800D0058037BD01291AD17D
:10762000FFF76AFF041EF8D001235B420380A378B2
:10763000FF2BF2D0FE2B07D00023E078142200931A
:1076400029001E3300F032FBA01C00F053FB012385
:107650005B426380E1E70229DFD1013901F0BEF826
:107660000028DAD12800FFF747FF041EDFD1D4E756
:10767000FEFF0000FFFF0000022210B5074B524240
:107680001A80074801325A809A80DA8000F07EFA28
:10769000044801F025F8002010BDC046E864FF1F33
:1076A0001D750011F97500110388F7B50400002B52
:1076B00002D102252800FEBD426802211378254828
:1076C0005268FEF7A5FD00282ED0234F01253A88E9
:1076D000002AEFD0802321885B0201259B1A994262
:1076E000E8DC0C2004F0C4F8061E31D03B88228868
:1076F0009C4600231800019561469DB2491989B244
:10770000AA421BD8002801D062443A8000233000EE
:10771000082208C0210003F0D3FE104A1368002B92
:1077200013D100251660C5E76268022113780C4862
:107730005268FEF76DFD0028C7D1BAE760681D01E9
:107740004019418101330198D6E71A001B68E6E72A
:107750001325AFE7D2BC00112A43FF1FE464FF1FCB
:10776000D0BC0011014B18707047C0462C43FF1F5E
:1077700014230A0010B51A40194204D00122102126
:1077800001F048F810BD4B06F9D4012088434000B1
:10779000F8E710B514008B0604D50122102101F082
:1077A00039F810BD08230A001A40194202D14BB221
:1077B000002B0FDA102101F02DF8002808D023004B
:1077C000F2331B78002BECD0F1342378012BE8D175
:1077D0000020E6E703208907FAD4E2E7F0B51F00AE
:1077E000184B85B01C68019002910392002C27D1A0
:1077F000200005B0F0BDA5683301ED186B89019A32
:10780000934211D3029A93420ED8002F04D10A9BBF
:10781000002B10D12C00EBE73B002978039A686815
:10782000FEF7F6FC0028F2D10136B6B2A388B342C7
:10783000E1D82468DAE7A3680A9A5B891380E9E74C
:107840000026F3E7E464FF1F37B50C000A88498877
:107850000123914217D3002A15D0651D23792A00F0
:1078600002210A48FEF7D4FC102300280BD023790C
:107870006188208800242A000094FFF7AFFF0A23C4
:10788000A04200D0230018003EBDC046D2BC00116B
:1078900013B50A0008884988012388420BD80028BC
:1078A00009D00024137905320094FFF797FF0A23CB
:1078B000A04200D02300180016BD13B50A000888A6
:1078C0004988012388420BD8002809D00024137965
:1078D00005320094FFF782FF0A23A04200D0230064
:1078E000180016BDF0B58BB003904A8808880E00CA
:1078F0000123824255D3002853D00023012704AC32
:1079000023700022718813000092FFF767FF051EA5
:107910003ED02078002835D12B78022B18D1677003
:107920006A8983000130E31880005A806968022266
:10793000201803F0C5FD23780133DBB22370042B3C
:1079400019D93B006889013080B2002BD9D01FE0E3
:1079500002236370122358436A89231804305A8023
:1079600069681022201803F0ABFD23780133DBB2E5
:107970002370002BE5D10C4A6B899B185A42534166
:10798000DBB2DFE76378012BE4D12B78022BC7D081
:1079900022780A23002A04D021000398FEF798F9E0
:1079A000002318000BB0F0BD0100FFFF0F4BF0B536
:1079B00004001868002816D083685D89A54207D89E
:1079C0008288AE18B44203DA12019A18934201D1A8
:1079D0000068EFE71E005F891036A74204D1002936
:1079E00000D00D801800F0BD3300EFE7E464FF1F06
:1079F00070B505000C0008880021FFF7D7FF0300D1
:107A00000120002B04D022002800197AFFF7C1FEC4
:107A100070BDF7B50C00002501902300EE331B78F4
:107A2000AB4201D800200AE06B00E65A002130008A
:107A3000E718FFF7BBFF002802D126800130FEBD0A
:107A4000017A0198FFF794FE002802D03B8823803A
:107A5000F5E70135EDB2E0E710B504000888002134
:107A6000FFF7A4FF03000120002B03D02000197AA8
:107A7000FFF77EFE10BD0000054B1B68002B01D1F7
:107A8000180004E09A6852898242F6D198887047BB
:107A9000E464FF1FF0B50E27002687B0039302AB06
:107AA000FF183E8005001F4B40891400984207D004
:107AB0002B78013000976A6880B2FFF78FFE0600CE
:107AC00002212B7818486A68FEF7A2FB00280FD025
:107AD0006C892000FFF7D0FF002802D0013C041978
:107AE000A4B2039B002B00D01C80300007B0F0BD77
:107AF00002212B780D486A68FEF78AFB0028E7D13F
:107B000002212B780A486A68FEF782FB002807D01A
:107B1000002EDED03B88A342DBD17489013CDFE735
:107B20006C89DEE7FFFF0000D2BC0011D0BC001161
:107B3000CEBC001110B50C00FFF7DEFC03000220E4
:107B4000002B0AD0002C00D023609B781720FE2B3E
:107B500003D00138FF2B00D1002010BD73B50D00FC
:107B600001A904001600FFF7E5FF172805D0002E35
:107B700004D129002000FEF727F976BD012210214B
:107B8000200000F047FE0028F3D0F6E7014B186014
:107B90007047C046F464FF1F37B56B469D1D01005A
:107BA00004000222280003F033FE2B88B02B0ED1F4
:107BB0002379122B09D12300FA331B78012B06D12C
:107BC0000121608800F0E0F801E01B2BF8D037BD00
:107BD00010B5054B0421187000F098F8FFF74CFD24
:107BE000FEF770FB10BDC046F864FF1F0020F0B523
:107BF0000BB20F0087B0834234DA274B187803F0BA
:107C00009FFE051E2BD00378A02B25D103AE31009B
:107C1000FEF7E4F8041E0BD1B378DB0724D51F4B25
:107C200006341B68002B03D0310068889847040095
:107C3000A868002801D003F063FC002C08D1184A82
:107C4000039B1340174A934206D0B3781B2B03D0F3
:107C50000121688800F098F8280003F011FE8020C8
:107C60000002784007B0F0BD0F4B1B68002B10D00E
:107C7000310068889847041EDAD07378002BD7D17A
:107C8000B27801A90A704B800C716888FDF7F6FF85
:107C9000CEE70624F1E7C046F864FF1FF064FF1F3B
:107CA00000FFFF0000011200F464FF1FF7B5019010
:107CB000FC200D0017001E0003F012FE040013202C
:107CC000002C12D0B02320002370089BF422677090
:107CD000658026710830002B08D0190003F0F0FBF6
:107CE0002100019803F0DCFD0020FEBD089903F09F
:107CF0000FFCF5E710B5041E06D00078FD2803D868
:107D000003F056FBFF23237010BD00000A1F93B23F
:107D100010B504000220032B05D882400020024B3E
:107D2000D1529B189C7010BD1865FF1F0B8870B551
:107D3000043B04000D000220032B0BD8012120007E
:107D400000F04CFD03001420002B03D0290020007C
:107D500000F0DEFB70BD000007B51300034A00927F
:107D60000A00012100F02CFC0EBDC046957F0011D9
:107D700007B5019203220092024B0A00122100F083
:107D800049FC0EBD1380001107B56B4601AA118096
:107D90000449D88008780633012802D1190003F07D
:107DA000C7FB07BDF964FF1F0C4B10B5187000230B
:107DB000FF210B4A1380138193819380094A5380DA
:107DC0001370517293819372D174D382137551776A
:107DD00003F07EFC00F0FCF910BDC0462865FF1FD3
:107DE0001865FF1FFA64FF1FF0B58DB06B460020C9
:107DF00003910C229B5E834200DBB0E05D4B187860
:107E000003F09EFD051E00D1A4E00378902B00D066
:107E10009DE006AF01004688380000F013FA79684B
:107E20000400002900D19CE03B88052B6ED13B89E2
:107E3000032B1CD905AC200000F0A2F86288172A99
:107E400061D83989131D994231D179682378043179
:107E50000291D90738D5607800F08EF9071E06D058
:107E6000002303712378012B08D0132B23D0A8689B
:107E7000002800D178E003F043FB75E062880299A6
:107E800009A800F0A6F80290380000F08BF909AAC2
:107E90002378387A0192002231000092029A00F091
:107EA00012F9380000F064F9029B002BDFD030009B
:107EB00000F080F9DBE70378032BD8D162880299C0
:107EC00009A800F0D6F8DEE7122B13D1029909A811
:107ED00000F0B5F8021EEAD127498B88002BC6D0E6
:107EE000887909A92378019161780091310000F027
:107EF000EAF8BCE7002302AA93833000617809AA5C
:107F0000FFF72AFFB3E71D4B0993F6E7042B02D0D6
:107F10009A1F012AABD8184A043B9B00995A0029A2
:107F2000A5D0D218907831003A0000F0AEF80028C1
:107F30009DD13B88042B03D001213000FFF724FFA3
:107F4000012C04D1A868002801D003F0D9FA280038
:107F500003F096FC8020039B0002434018000DB004
:107F6000F0BD012800D182E701213000FFF70CFFAE
:107F7000EDE7C0462865FF1F1865FF1F01001700C9
:107F80000B7803704B784370CB788A781B021343CD
:107F9000438070470A88030002700A88120A427000
:107FA0000A88012A06D14A8882704A88120AC27059
:107FB0000420704702208242FBD14A8804309A7024
:107FC0004A88120ADA708A881A718A88120A5A71E3
:107FD000EFE710B50400012082420CD94B780A78F3
:107FE0001B0213432380834206D1CB788A781B027D
:107FF00013436380002010BD022BFBD1CB788A781D
:108000001B02134363804B790A791B021343A3803D
:10801000F0E70B8803700B881B0A43704B88837052
:108020004B881B0AC3708B8803718B881B0A4371B2
:10803000CB888371CB881B0AC3710820704703006B
:108040000120082A14D14A780878120202431A80C3
:10805000CA788878120202435A804A790879120253
:1080600002439A80CA798879120202430020DA809A
:10807000704710B504000120022A05D100204B787A
:108080000A781B021343238010BDF8B506001020A8
:108090000F00150003F024FC04000120002C0ED07A
:1080A000A0230C22290023806780201D002D07D0EB
:1080B00003F006FA2100300003F0F2FB0020F8BDC7
:1080C00003F026FAF6E7F7B51E00009008AB14207F
:1080D00017001D78019103F003FC041E12D0A223A7
:1080E0000370019B47704380099B057146710C2208
:1080F0000830002B07D0190003F0E2F921000098A6
:1081000003F0CEFBF7BD099903F002FAF6E737B5A5
:10811000041E0FD04388002B0CD00025C1881323E8
:10812000007A172201950095FFF7CDFFFF236580A8
:108130006372257037BD000010B50C4904004A88F1
:10814000002A09D08B89002B05D00020CB8A02227F
:10815000834201D010BD012213000A2043430020B6
:108160004032C854C81842800472F3E7FA64FF1F13
:108170000023438003707047094B00211A0010B59B
:108180005C88002C06D01C79844203D10A234B431F
:10819000D01810BD01310A330329F1D10020F8E7CE
:1081A000FA64FF1F10B50400407A03F001F9FF23C1
:1081B000637210BD7047043010B580B203F010FB3D
:1081C000002803D00421494203F0D2FA10BD000078
:1081D00070B50025104CA0682580A581A580A84217
:1081E00002D003F08DF9A56000250C4C0C4B606D9E
:1081F0001D80230058331D70A84202D003F080F97F
:10820000656500256068002801D003F079F9013523
:1082100008340A2DF6D170BDC065FF1F6465FF1FCD
:10822000B465FF1F70B5041E09D1054D2880A881D3
:10823000A880A868002802D003F062F9AC6070BD85
:10824000C065FF1FF0B54B8885B0019300234360E4
:108250000A7905000F00022A00D07BE0CA88032AB1
:1082600017D98B685E7819783602DC78D8790E4396
:1082700099781B7A24021B020C43034353495BBACF
:108280000B80331D93421ED1042C04D0631F022B9C
:108290000ED9012015E0019A4D4B1201D35A002B43
:1082A00006D00198FFF7BEFF4A4A136901331361F4
:1082B0000421B8682E812C80494203F059FA686085
:1082C000002005B0F0BD434D042C06D0631F022BE7
:1082D0000FD9EB680133EB60DBE7019A3C4B1201ED
:1082E000D35A002B05D00198FFF79CFF2B6901336F
:1082F0002B61374B30000293019B029A1B010193C3
:10830000002301998C468B52130063449C80039395
:108310009E81FFF750FF039B041E986016D0042136
:10832000B868494203F024FAFA880100043A2000B0
:1083300003F0C6F80199029AFB888A5A043B9B18FD
:10834000029A8B522B6801332B60A2E7AB69013391
:10835000AB619EE71E4B0293019B1E01029BF35AE9
:10836000002B2DD002998C19A068002828D0012A52
:1083700026D1FA889B189BB27352A189994217D3D0
:108380009B1AC018B96803F09BF8029BA289F35AA4
:10839000934200D07DE700222B81A3882B80A36825
:1083A0006B60029BF2520B4A53680133536070E7D3
:1083B000084A9368013393600198FFF733FF68E739
:1083C000044A536901335361F6E7C0462A65FF1F2B
:1083D000C065FF1F3065FF1F70B5051E15D10B4C22
:1083E0000B4B1880230058331870606D002802D0A2
:1083F00003F086F86565250050356068002801D0D7
:1084000003F07EF80834AC42F7D170BD6465FF1FFD
:10841000B465FF1FF0B51700A12285B0920001934B
:108420004243394B06001B680C009B18D933FF33BD
:108430001D78FDF741FF0430854204DD3000FDF773
:108440003BFF0430C5B2BD4207D33A0000213000E3
:10845000019B03F09DFA05B0F0BD2900380003F040
:10846000CFF92300C6B250331E700393019B29003D
:108470006365380003F0ACF8CBB20293002B02D056
:10848000039B01361E7000262300503303931B7894
:10849000B34204D8606D002831D10020DBE7029A96
:1084A0002800002A04D0013B1000B34200D028006D
:1084B000F700E719387003F07BF8786000280ED0D9
:1084C0003A78019902F0FCFF019A3B780136D31803
:1084D0000E4A0193D369F6B20133D361D4E7039B0B
:1084E00018706065A74205D1084A1320D36A01338A
:1084F000D362B0E7606803F003F80834F2E702F0F3
:10850000FFFF00236365C8E73409FF1F3065FF1FC5
:10851000F7B50D0007000421686803F029F92B89DD
:10852000040003702B891B0A43702B8883702B88EF
:108530001B0AC3702E8902250436F6B2F42E15D814
:108540001B4B9F4214D10C2003F0CAF91135011EB8
:108550000CD0902303708E3B0371043B4380154B7A
:108560008460C680187803F09BF900252800FEBDC2
:108570005C237B43104AD3180093583301931B7834
:10858000002B0FD10300320038000099FFF742FFA3
:10859000019B05001B78002BE8D13800009902F000
:1085A0001FFFE3E7054A0725536A01335362DDE7FE
:1085B000FEFF00002865FF1F6465FF1F3065FF1F79
:1085C000F0B587B0009017200F0016000193FFF759
:1085D000F2FD1325041E19D00C98031E02D0019938
:1085E000201D9847030AE370052302AAA0700430F7
:1085F000908127700098667003A993800494FFF718
:1086000087FF051E02D0200002F07AFF280007B085
:10861000F0BD0000F0B587B01F000CAB1B780391D4
:10862000059301210DAB06001C78049200F0D6F8EA
:108630001425002821D02000FFF77EFD0135041EFF
:108640001BD01149059B0A7803700132D2B2131E68
:10865000C68001D101231A000B7022713000049BE7
:1086600003990097FFF7ACFF051E09D123002100F5
:108670000648074A093302F06BFF280007B0F0BD37
:10868000002363802370F8E72C65FF1F0F81001122
:1086900030750000F8B505000E00064C064F236843
:1086A000002B02D03100280098470434BC42F6D198
:1086B000F8BDC046D065FF1FE465FF1F0123064AD1
:1086C0005B425380002313715362044A136053606A
:1086D0009360D36013617047E465FF1FD065FF1F8F
:1086E0000200002310B506499C000859002801D15A
:1086F000625010BD0133052BF6D11320F9E7C046B7
:10870000D065FF1F034A5388181A4342584140421C
:1087100010407047E465FF1FF0B585B002930AABC7
:108720001F780CAB1B88009008000E000192039389
:10873000FFF7E8FF05001120002D1BD10E48FFF7C1
:10874000E1FF04001520002C14D006220B99A7711C
:10875000E01D02F0B5FE019B30002371029B290051
:108760006371009B66802370039B6562E381FFF762
:1087700091FF280005B0F0BDFFFF000010B5FFF726
:10878000C1FF04000220002C12D060880121FFF7F5
:1087900081FF606A002801D002F032FE2822002109
:1087A000200002F0B5FE012300205B4263802071AF
:1087B00010BD000030B5074A074C558801001378FA
:1087C0000020A54204D05B1A59424B415842104048
:1087D00030BDC046E465FF1FFFFF0000084A10B52A
:1087E00001230C00904208D0FFF78CFF031E04D039
:1087F000037923405A1E9341DBB2180010BDC046D6
:10880000FEFF0000024B1879431E9841C0B270472A
:10881000E465FF1F70B504000D001600FFF772FF3E
:10882000002804D10D4B9C4200D0143070BD416A29
:1088300003790520002907D012221A40102A02D1FC
:108840000520002EF2D10F20DB06EFD5897E0C200B
:10885000A9428941494249420840E7E7FEFF00003A
:10886000030010B5002800D110BD0348034A418819
:108870009142F9D09847F7E7E465FF1FFFFF00003A
:10888000002330B5C45CCD5C6C40D4540133102B54
:10889000F8D130BD0F23002210B5C45C6400224320
:1088A000CA54C25CD209013BF7D210BD02000100DC
:1088B00010B52032103103F02BF810BDF0B58BB09D
:1088C0000390102005931700049102F0D1FF00904F
:1088D000102002F0CDFF009B13240190002B05D047
:1088E00000280CD11324009802F08AFD019B002B74
:1088F00002D0180002F084FD20000BB0F0BD102063
:1089000002F0B6FF0600102002F0B2FF13240500AB
:10891000002E00D1AEE0002819D01022002102F074
:10892000F7FD32002900039802F0F2FF041E0ED179
:1089300033787F2B51D830000099FFF7ABFF009BB5
:108940001B787F2B53D801990098FFF7A3FF3000C5
:1089500002F056FD002D02D0280002F051FD002C3F
:10896000C1D1102002F084FF0600102002F080FF29
:108970000290002E7CD0002878D03A000F322300DD
:108980000125121105D00F333B4015B25A42534115
:108990001BB26A1E1201002B33D0049BD2B298186E
:1089A0000099029AFFF76CFF013D10220021300070
:1089B00002F0AEFDADB2049F2D017D19AF4242D051
:1089C000002C33D0300002F01BFD029B002B00D1A5
:1089D00089E7180002F014FD85E729003000FFF751
:1089E00059FF28002549009AFFF74AFFA7E7290009
:1089F0000098FFF74FFF28002049019AFFF740FF3A
:108A0000A5E70F210F4004998A18D9B28F4208D9DF
:108A1000D15C06A819540133102BF6D1029A0199A2
:108A2000C0E7791A48424141C901F2E739003000F4
:108A300006AAFFF725FF3200039806A902F068FF97
:108A400010370400BAE7002CBCD13000029906AA06
:108A5000FFF716FF320006A9039802F059FF08221B
:108A600004003100059802F02BFDABE71324A9E7C1
:108A70001324AAE7002800D06EE733E7D8BC001122
:108A8000F0B58BB00F0016000225009000283FD0F3
:108A9000002A3DD00B1DDBB21800029302F0E8FE65
:108AA0001135041E34D0FDF747FD05003A0000994A
:108AB000201D02F0A5FFEBB20393E3702B0CDBB299
:108AC0002F0A00936370FFB22B0E2370A7700193DF
:108AD000FDF72CFD1022010006A802F091FF2100F5
:108AE000029A04AB06A8FFF7E9FE051E0DD1039B11
:108AF00008223370009B04A9B370019B7770F37058
:108B0000301D02F07DFFFDF71DFD200002F078FC16
:108B100028000BB0F0BDF0B58FB00D00149E03908F
:108B200004920593002A03D1022420000FB0F0BD67
:108B3000002EF9D00398FFF7E5FD1424071EF4D0AA
:108B40007278337812021A43B3781B041343F27815
:108B500012061A43036A0192934201D30133E3D10F
:108B6000002D03D03B7901249B07DED5082200218C
:108B700006A802F0CDFC059B13240433DBB21800D9
:108B8000029302F075FE051ECFD0059A04990430B9
:108B900002F036FF04223100280002F031FF3900D4
:108BA000102210310AA802F02BFF2900029A06AB0E
:108BB0000AA8FFF783FE041E0FD1082206A908A801
:108BC00002F01EFF0822311D08A802F011FD012845
:108BD00007D101990398FDF7C9FC280002F010FCA9
:108BE000A3E70124F9E7000070B51C4C05002368D9
:108BF000181E10D0002D14D11A78002A0CD1981C00
:108C0000083202F05DFC02F0E3FE0135002808D1D5
:108C100023681D70012070BD0A331800082202F07D
:108C20004FFC2368002BF5D0122002F059FE061EDF
:108C30000DD0C1232168037045700231102202302B
:108C400002F03EFC23683100587802F029FE2068CB
:108C500002F0D6FB00232360DCE7C0460C66FF1F52
:108C6000F8B504002020FDF755FB0D4EA700BB59B9
:108C70000500002B0DD000280BD0D878FF2809D193
:108C800008492A000C55F35907480333611802F0CC
:108C90005FFCF8BD290002F0D3FD0028F0D1F8E711
:108CA0002866FF1F1066FF1FB99E001170B5064DA4
:108CB00084006359002B05D0D87802F079FBFF229D
:108CC0006359DA7070BDC0462866FF1F70B5060094
:108CD0008CB00C00150000213022684602F018FC10
:108CE00031001022684602F08BFE1D202100032275
:108CF000684402F085FE6846FFF7D8FD2D21040088
:108D000003222800694402F07BFE20000CB070BDF5
:108D1000F0B50700160097B001931CAB1D78302208
:108D20001EAB00910AA800211C7802F0F1FB102272
:108D300039000AA802F064FE1022002102A802F005
:108D4000E7FB0722310002A802F05AFE072202AB1D
:108D50009818631E9C41019902F052FE02AB9C736D
:108D60002B005A1E934102AAD3730021102206A899
:108D700002F0CEFB06221D9907A802F041FE1A2040
:108D800002ABC01806221F9902F03AFE1022009989
:108D90000EA802F035FE102202AB0EA908781C784E
:108DA000013A6040D2B2087001330131002AF5D196
:108DB0000AA8FFF77BFD102212A904000EA802F0FA
:108DC0007FFB102206AB0EA908781D78013A684097
:108DD000D2B2087001330131002AF5D10AA8FFF799
:108DE00065FD044310222098E4B212A902F008FEA7
:108DF000200017B0F0BD70B50E0014008CB001005B
:108E0000102268461D0002F0FBFD3100082204A874
:108E100002F0F6FD2100082206A802F0F1FD6846E6
:108E2000FFF744FD04001022280008A902F0E8FD25
:108E300020000CB070BDF8B506000D0000243719F5
:108E4000AC4200D3F8BD02F053FB030A3B70631C35
:108E5000DBB201379D4203D90234F054E4B2EEE7AD
:108E60001C00EDE773B506000C000225002819D0A0
:108E7000002917D0032101A8FFF7DDFF6B469A797F
:108E80003F231A40013313436A463000937101A90E
:108E90002200FFF71BFF051E04D10322E01C01A9DD
:108EA00002F00EFB280076BD03785807DA08C00FE1
:108EB000D20080009B0710439B0F1843C0B270473D
:108EC00007230B40C908C9000B430370704700001B
:108ED00070B50400FFF7EAFE134DA4006359002BA0
:108EE00021D0186A002801D002F08AFA2B59986E16
:108EF000002801D002F084FA2B59D86E002801D046
:108F000002F07EFA2B59186F002801D002F078FA8F
:108F10002B59586F002801D002F072FA285902F03C
:108F20006FFA00232B5170BD2866FF1F0E4B800087
:108F3000C35870B50C00002B0FD09D68002D0CD0CD
:108F40002B78201D0B706B784B70A97CFFF7B8FF56
:108F50002B7E23726B69E36070BD1022002120001C
:108F600002F0D6FAF8E7C0462866FF1F014B1860EA
:108F70007047C0462466FF1F074A030080008258DE
:108F800010B5002A06D0D088984203D1012901D11A
:108F9000FFF79EFF10BDC0462866FF1FF0B5264EA6
:108FA00095B087000B93BB590500099112200A92D6
:108FB000002B31D0D888FFF7A5FB04001420002C2B
:108FC0002AD0280010A9FFF7B1FFBB591E781D6AEF
:108FD000002E23D00895FDF7EFFA07000020FDF7DB
:108FE000F1FA0790A379E61D069310AD0CA9089835
:108FF00000F0E2FA0EA9280000F0D7FA0B9B0A99BC
:109000000493069B09980293079B0396019300978C
:109010000EAB0CAAFFF77CFE15B0F0BDFDF7CCFA45
:1090200006903000FDF7CEFAE31DA779079310AB49
:1090300006000893DAE7C0462866FF1F30B50C4CDF
:1090400085002A59030085B00120002A0ED018009F
:109050006946FFF76BFF2B591A78D888054B002A11
:1090600000D1054B6A46072100F0D9FB05B030BDA1
:109070002866FF1FAB950011B995001130B5094C5A
:109080008500295985B010226846253102F018FA6A
:109090002A591121044BD0886A4600F0C0FB05B064
:1090A00030BDC0462866FF1F5596001130B5094CEB
:1090B0008500295985B010226846353102F000FA42
:1090C0002A591121044BD0886A4600F0A8FB05B04C
:1090D00030BDC0462866FF1F93960011F7B54D4F6F
:1090E00086001020F4590D0002F0C2FBF3592062F3
:1090F000186A132200286CD0033A29009C6802F0F9
:10910000DFF9F3591A780192002A58D11E6A227D9C
:10911000317B944651400122019F114201D16746A3
:109120001740217D914339432175377B4F40BC4621
:1091300060460027800701D44F0817400121022014
:109140008F40227D82433A432275377B5740BC468D
:1091500060460027400701D497080F400420227D75
:10916000BF0082433A432275627D002794466046E1
:10917000727B42400A4201D167460F400121627D65
:109180008A433A436275777B5740BC466046002766
:10919000800701D457080F400220627D7F00824380
:1091A00017436775767B00227E40760701D4BA08A4
:1091B0000A400426617D9200B1430A4362756A78D1
:1091C000002A08D06278002A05D005220533DA7714
:1091D00000221000FEBD04222979114205D1A17C94
:1091E000114202D10533033AF1E7019A21782C7834
:1091F000002A02D10A002100140018220429E8D80C
:10920000042CE6D805206043034A05331218525C4B
:10921000DDE7C0462866FF1FE8BC001110B50A0054
:109220001121024B00F0FBFA10BDC046EF96001171
:109230000B0030B587B001AD2B806B4604001100E8
:10924000981D082202F03CF92A000B212000024B55
:1092500000F0E5FA07B030BD1797001110B50A000D
:109260001121024B00F0DBFA10BDC0466B970011D4
:1092700013B50B0011006A4613706B4604000622FA
:10928000581C02F01DF96A4608212000014B00F02D
:10929000C6FA13BD8B97001110B50A001121024BBD
:1092A00000F0BDFA10BDC046DB9700117FB5050088
:1092B0000B4BAA00D4580800002C0FD0666F237FF8
:1092C000E28821780396266F0296E66E0196A46ED8
:1092D0000094FDF709FC2800FFF7FAFD7FBDC046AA
:1092E0002866FF1F10B51721FFF7E0FF10BD000033
:1092F00070B50A000D00064B0221040000F08FFA41
:10930000060029782000FFF7D1FF300070BDC0466D
:10931000BB96001170B586B000236A46137083684F
:1093200004001D78681E0A2859D801A902F098F98E
:10933000060633373B3F43474B4F5300180000F0BE
:1093400042F9062312284BD000281BD16088FFF772
:10935000D9F90823002813D04279002A47D1264B97
:109360001A78072312070BD5244B1A680723002A03
:1093700006D01668002E03D0290001AAB0470300CA
:109380006A4613706B461B786088002B2AD1FFF762
:1093900067FC06B070BD180000F06CF9D4E7180047
:1093A00000F087F9D0E7180000F093F9CCE7180037
:1093B00000F0ADF9C8E7180000F0C3F9C4E71800E1
:1093C00000F0F6F9C0E7180000F0F6F9BCE7180065
:1093D00000F013FAB8E7180000F013FAB4E7072317
:1093E0006A46137069466088FFF782FFD1E705235C
:1093F000012AC5D1024BB8E7B564FF1F2066FF1FE5
:109400002466FF1FF8B52C4F8600F35904000D00A9
:10941000002B40D0DA8882423DD15A78062A33D1D7
:109420001A78002A2ED0012099681A6A097D014213
:1094300006D0157B054203D007225A700120F8BDE3
:109440000220014204D0157B054201D00922F4E735
:109450000420014204D0127B024201D00B22ECE72F
:10946000164B1B68002BE9D05B68002BE6D0200070
:109470009847BB5900215B78122BDFD12000FFF702
:1094800015FFDBE70E4BECE7112A04D1002900D0D1
:1094900032252900F2E7002D08D12000FFF732F92C
:1094A000002803D010230279134303712100280000
:1094B000FDF798FAC2E7C0462866FF1F2066FF1F27
:1094C0002466FF1F70B50E4E8500AB590400002BBB
:1094D00013D01B78002B11D10A4B1B68002B04D032
:1094E0005B68002B01D02000984773595B78122BE2
:1094F00003D100212000FFF7D9FE70BD024BECE73D
:109500002866FF1F2466FF1F2066FF1F094B80008F
:10951000C3581020002B0CD01A6A002A09D09B686F
:10952000002B06D0127A1B7E101C9A4200D9181C00
:10953000C0B270472866FF1F70B503000D0014000D
:109540000220002A30D000292ED013700B78081D7D
:1095500053704B789370FFF7A7FCE0700120022155
:109560002B7A23716B7B034063716A7B0A40134340
:10957000042263716E7B1640334363716E7BF60881
:10958000F600334363712B7B0340A371287B0140BA
:1095900000200B43A371297B0A401343A3712A7B4C
:1095A000D208D2001343A37170BD10B50A000100A8
:1095B0000120FFF7C1FF10BD10B50A000100022015
:1095C000FFF7BAFF10BD70B506000C000220002E98
:1095D00030D000292ED07378201D0B70B3784B70DB
:1095E000F178FFF76DFC01223579257271794B1006
:1095F000080013409340104003438810104080003F
:10960000C9080343C9000B436373B1794B100800C9
:109610001340934010400343881002409200C90851
:109620001343C9000B4321202373FCF773FE8542CB
:1096300001D2122070BD2220257AFCF76BFE8542F4
:10964000F7D823781820042BF4D86378012BF1D8AD
:109650000020EFE7030010B50220002909D0002BFD
:1096600007D00322481C0A7019000D3201F028FFB0
:10967000002010BD03000222080010B5002B06D008
:10968000002904D00E32591C01F01AFF00221000EC
:1096900010BD030010B50220002909D0002B07D00F
:1096A0000422481C0A7019000C3201F009FF002046
:1096B00010BD10B5FFF7DEFF10BD0300022000292A
:1096C00006D0002B04D0052200200A701B784B70B6
:1096D000704703000220002B08D0002906D05B78D9
:1096E00000200B70013B082B00D918307047030095
:1096F00010B50220002909D0002B07D00622481CF3
:109700000A7019000A3201F0DBFE002010BD10B50E
:10971000FFF7B0FF10BD02000B00022010B50029BA
:109720000ED0002A0CD007211970118859701188A9
:10973000090A997011180822D81C01F0C1FE0020F6
:1097400010BD03000A00022010B5002B0CD0002928
:109750000AD099785878090201431180901CD91CCD
:10976000082201F0ADFE002010BD030010B502205C
:10977000002909D0002B07D00822481C0A701900C4
:10978000921801F09DFE002010BD02000B00022087
:1097900010B500290BD0002A09D0092119701178C1
:1097A00018185970511C062201F08AFE002010BDC5
:1097B00010B5FFF75FFF10BD02000B00022010B5CF
:1097C000002A09D0002907D05178197011180622F3
:1097D000581C01F075FE002010BD030010B50220DA
:1097E000002909D0002B07D00A22481C0A70190052
:1097F000063201F065FE002010BD10B5FFF73AFFFC
:1098000010BD02000B00022010B5002A06D000296E
:1098100004D018005178FFF753FB002010BDF0B5BD
:1098200085B017001E006A460623050008009181D6
:109830009380FEF7C0FC1324011E02900CD0380068
:10984000B047041E05D1280001A9FEF76FFA041ED7
:1098500002D0029801F054FE2800FFF701FA200020
:1098600005B0F0BDF0B504008BB0019115000021EA
:10987000102202A801F04CFE334EA700B859002870
:109880003CD0C388A34239D10378002B36D142782B
:10989000062A18D102000100553235310C3006ABD2
:1098A000FFF7A9FA002829D12000FFF72FFE0200B8
:1098B00006A902A801F004FE200002A901F068FE3A
:1098C00001200BB0F0BD816E002917D00B8A112A40
:1098D00028D19D420ED101981231093A01F088FE3B
:1098E000012807D1BB5920009D6EFFF70FFE29000C
:1098F0000200DEE732212000FFF7D8FC2000FEF74F
:1099000001FF061E1BD0416A002918D00B8AAB420A
:1099100015D108220198123101F06AFE01280ED1FA
:10992000716A0AE09D42E9D108220198123101F0E2
:109930005FFE0128E2D1BB59996E8A7EB9E720000B
:1099400001F00EFEBCE7C0462866FF1FF0B56B4D68
:1099500087007E5985B0337802900393002B00D0A6
:1099600087E0B368346A01937078062817D1012222
:109970001B7D134202D0217B114218D102221342D7
:1099800002D0217B114251D10422134203D0237B08
:10999000134200D08BE0019B5A7DEB5991E00738D0
:1099A0000428F8D801F05CFE032E42678300B36EF2
:1099B000002B03D11C2001F05BFFB066EB599C6EBD
:1099C000002C1CD010220021200001F0A1FD0298E3
:1099D000FFF79CFD01002000FFF72DFA01F088FD44
:1099E0002082200008211230FFF725FA0298FFF7A5
:1099F0008DFDA076EB592100D888FFF70FFC0822D7
:109A0000EB591CE0B36E002B05D01A00198AF088C0
:109A10001232FFF70DFC0222019B197DEB59114216
:109A20003DD0207B10423AD0073208E0F488FCF7A2
:109A3000DBFD01002000FFF711FC0A22EB595A70F0
:109A4000029B9C002A595378073B042B11D8D088DD
:109A5000FEF758FE00284ED0C3895A08D21828496C
:109A6000029B0298CB542B5941180433254801F02E
:109A70006FFD05B0F0BDFCF79FFD030001208342A0
:109A800001D100200393EB59DE88FCF79BFD03997D
:109A900002003000FFF7ECFB019AEB59117D042224
:109AA00011420CD0217B114209D00B22C7E7F68866
:109AB000FCF73CFD01003000FFF7EEFB6BE7019A7D
:109AC000527D01210A4204D0607B084201D00C2261
:109AD000B5E702210A4204D0607B084201D00E2281
:109AE000ADE704210A4204D0627B0A4201D0102271
:109AF000A5E71222A3E7FA225200B0E72866FF1F6B
:109B00002C66FF1FC39E001110B5064B1A78042364
:109B1000100018401A4200D00348FFF727FA00202F
:109B200010BDC046B564FF1F3043FF1F70B5040071
:109B3000FFF7D4FA051E43D12000FFF77FFA234E2A
:109B4000A400A0598268937CDB0708D50321036A2F
:109B50001B790B40012B02D1017F0B430377431D7F
:109B6000D97F8B1E022B0DD8022900D00121C0887D
:109B7000FCF790FF042133591A7F59700A431A7772
:109B8000280070BD01290CD102231022437000214E
:109B90000C3001F0BDFC305910213530FFF74BF986
:109BA000EEE70529ECD10223D118437010220C30C6
:109BB00001F086FC04233259117F0B431377EAE747
:109BC00008251828DCD1053DDAE7C0462866FF1FC6
:109BD000F0B58BB0059143887E4F9E00F459150077
:109BE0000493002C15D1012902D000200BB0F0BD48
:109BF000101D57781678FFF757F9EB68320002937B
:109C00002B7A0499019300903B002000FCF70CFF95
:109C1000EBE7E388049A934201D00820E6E7237833
:109C2000012B00D1D4E0059B581E092800D9CFE0B4
:109C300001F016FD05CE0A29CC506C859AB2290098
:109C40000498FFF773FFD1E7200029001022453068
:109C500001F036FCB9594B78042B02D1013B4B7013
:109C6000C3E70B000A00253335320C310498FFF7A7
:109C700095F90498FFF702FA0522431E9841BB5953
:109C8000C0005A70B2E7200029001022553001F0C0
:109C900017FC049B4F4C9D00295904980A0006AB01
:109CA00055320C31FFF77AF929591022453106A8AF
:109CB00001F09EFC012808D10498FFF7F7F9059000
:109CC000002804D106222B595A7005988EE70823E4
:109CD0000593FAE763780C2B7AD1E36E002B03D15E
:109CE0001C2001F0C5FDE066BB59D86E00286FD07E
:109CF0001022290001F0E4FBBB590498DC6EFFF749
:109D000005FC0D22A076BB595A706EE7E06E002864
:109D10005ED063780D2B5BD12B8808220382A91CAF
:109D2000123001F0CDFBBB599A68517D02221142DD
:109D300026D0186A407B104222D00C32E4E76378C8
:109D40000E2B45D1236F002B03D1162001F090FD7F
:109D50002067BB59186F002803D01022290001F09A
:109D6000AFFB0F22BB59CFE763780F2B30D1206FA9
:109D70000622691C103001F0A3FBBB599A68517D83
:109D80000422114203D0196A497B1142D5D1002126
:109D90000498FFF78BFA28E7636F002B0DD0BB59AF
:109DA000586F0028F3D01022290001F089FB01220E
:109DB000BB5952425B6F1A61E9E7142001F058FD6C
:109DC000BB5960675B6F002BE9D126E72978DFE795
:109DD00007200BE72866FF1F10B5064C207001F026
:109DE0006FFC06212078FDF791FF0348FEF778FC11
:109DF00010BDC0463B66FF1F798F001100200BB2DB
:109E000070B50D00834216DA264B187801F098FDE4
:109E1000041E0DD00378922B0ED0A02B37D0224BEE
:109E20001878FF283AD0210001F03AFD002835D1FA
:109E300080200002684070BD43780E2B0BD03E2B73
:109E4000EDD18378052B12D0082BE8D18179808859
:109E5000FFF7D8FA08E0154B82889A42DFD1836871
:109E60001878591CFEF7C0FE002817D1D7E7104B11
:109E70001B785B0712D50F4B1B68002B0ED09B681D
:109E8000002B0BD0C289811D80889847ECE7FFF733
:109E900041FAA068002801D001F032FB200001F057
:109EA000EFFCC5E73B66FF1F2943FF1F182000009A
:109EB000B564FF1F2466FF1F10B50078FFF712FA84
:109EC00010BD10B50078FFF7FDFA10BD0C23434319
:109ED000084A10B59B185A68002A03D0012901D1FD
:109EE000904710BD9B68002BFBD00029F9D1984703
:109EF000F7E7C0465866FF1F01238340094A10B5A3
:109F0000946B1C439463506B98435063D46B200054
:109F10009843012901D120001843D063116B0B43F2
:109F2000136310BD00800040F0B500240127154BDD
:109F300085B0DA6B144E03921A6C0192DA64019BBD
:109F4000E3403B4217D0039DE5403D400295E5B21A
:109F500002992800FFF7BAFF316A736A002908D016
:109F60003900002B01D0029979402800FFF7C4FF87
:109F700001E0002BF9D101340C36172CDFD105B0EC
:109F8000F0BDC046008000403C66FF1F064B01212B
:109F90005A68C2400A4204D01B68C34018000840F7
:109FA00070471B6DF9E7C046008000400122064B58
:109FB0008240002903D0D9680A43DA607047D96823
:109FC0009143D960FAE7C0460038004030B5032419
:109FD00044430F4BE25C1B199C785D7801232D1BD9
:109FE0000135AB40013BA340A140DB430C001228EC
:109FF00007D808499200521811681940214311608E
:10A0000030BD054A11680B4023431360F8E7C04692
:10A010002FBD001108F0004014F00040C21F70B5C1
:10A02000D4B20623092C0BD80125084C95400029F1
:10A0300008D00021FFF7CAFF23682B4323600023C9
:10A04000180070BD2368AB43F8E7C04600380040F5
:10A05000214BF0B51B185B78022B21D1032444431C
:10A060001E4A1F4EA35C12199478012215008540E8
:10A07000B76B013CE4B23D43A240B563194C1228D2
:10A0800015D89B0000290CD117495B1899680A4321
:10A090009A600123205C154A834011680B431360CA
:10A0A000F0BD11495B18996891439960F1E70E4B37
:10A0B00000290DD159690A435A61225C1328E8D05E
:10A0C0000123203A93400A49086803430B60E7E7FD
:10A0D000596991435961F0E73C66FF1F2FBD00119C
:10A0E0000080004074BD001100F00040A0F000406E
:10A0F000A4F00040F8B500241B4E1C4D1C4B1B5D0A
:10A10000012B1FD1194A9269E2401A420BD0012259
:10A11000B25693402200143AD2B2022A09D8154905
:10A120004A6913434B61013402360C35172CE5D1D3
:10A13000F8BD0022B2560F499200521891680B43A5
:10A140009360F0E7022BEED1E7B23800FFF71EFF75
:10A1500001235840C1B23800FFF77AFF3800FFF7FB
:10A1600015FF6877DFE7C04601BD00113C66FF1FA1
:10A170003D66FF1F00F00040012202388240054B7F
:10A18000002903D059690A435A61704759699143BC
:10A190005961FAE700380040F8B50E0001210F00C0
:10A1A0008740114A0400D368FD43BB43D360831E3C
:10A1B0008B4201D8FFF7E0FF00212000FFF72EFFC0
:10A1C0000A4A0B4B5168012E05D139431B195160C6
:10A1D0005E700020F8BD2940516002221C19627097
:10A1E0009A6915409D61F4E7003800400080004006
:10A1F0003C66FF1F012210B58240074B002906D0A4
:10A2000019680A431A600121FFF7C6FF10BD1968DB
:10A2100091431960F7E7C046008000400C2370B5F9
:10A22000002543430A4A29009B181D70094B04006E
:10A230001B185D70FFF7B0FF0123A34006492800FB
:10A240000A681A430A6005490A689A430A6070BDA1
:10A250005866FF1F3C66FF1F34800040308000407E
:10A2600070B504000E00FF2813D003250540FFF74A
:10A27000D5FF084AA3089B009B183F22ED00AA4087
:10A28000AE40196820009143314319600121FFF766
:10A290008DFE70BD18380040F8B50C244443134BB4
:10A2A0000500E4186368002B03D1A3681220002B7B
:10A2B0001AD0022201270E4B00215B195A70280088
:10A2C0002770FFF769FF63681E1E08D0A3683E0071
:10A2D000002B04D02800FFF759FE4640F6B22800B4
:10A2E0003100FFF709FE0020F8BDC0465866FF1F89
:10A2F0003C66FF1FF7B5C420FF222B4B8000195886
:10A30000002491433F3A0A431A508022274F5202B9
:10A31000274E1A60274B1D5D002D21D0A31E012B57
:10A3200003D80121E0B2FFF727FF012D18D11F4B01
:10A330009B69E3402B4213D0E3B218000193FFF76F
:10A3400025FE01000198FFF755FFE3B2143B022BF5
:10A350001DD801217156184A8D405369AB43536192
:10A360003B7F002B0DD0E5B22800FFF795FF2800BA
:10A37000FFF70CFE7B7F0100834202D02800FFF72D
:10A38000A5FD01340C370236172CC3D1F7BD0121CE
:10A3900000237156F3568D40074A9B009B189A681C
:10A3A000AA439A60DCE7C04600E100E03C66FF1F7C
:10A3B00001BD00113D66FF1F00F0004010B50121F6
:10A3C0000400FFF7E9FE0123044A002011194B7035
:10A3D000A34091690B43936110BDC0463C66FF1FCB
:10A3E00070B50E0015000400FFF718FF0C2363433F
:10A3F000094A20009B189D605E60FFF74DFFF02129
:10A40000064B074A8900051E5A5002D02000FFF76C
:10A4100005FF280070BDC0465866FF1F0000FF1FE3
:10A42000299F001170B5134D07202C78002C1FD1E7
:10A43000982221005200280001F012F80123C420C4
:10A44000FF222B700C4B80001C635C630B4B1C6069
:10A450005C600B4B195891433F3A0A431A508022D3
:10A4600052021A600D20074A074900F0F1FF200050
:10A4700070BDC0463C66FF1F00800040A0F0004059
:10A4800000E100E0F5A20011F5A00011030010B5F5
:10A490000620072B09D8054A137001F0A9F9D72126
:10A4A0000020034B034A89005A5010BD5843FF1F38
:10A4B0000000FF1F8D1BFF1F70B51D0002240C291B
:10A4C00010D8094ACA40D2070CD5FBF72FFF041E4B
:10A4D00008D1059A04992800FBF744FFFCF7B2FD68
:10A4E000FFF712FB200070BD1210000030B50D7890
:10A4F00002232C009C43184201D02B431C0008254A
:10A500002300AB43284201D02B00234320241D000D
:10A51000A543204201D01C4325002A230D70184278
:10A5200004D011781E3B0B43137030BD0028FCD1C2
:10A530000C2113788B43F7E7F8B51D0006AB1B8899
:10A54000140007AA0E000B201778002B27D10A78D9
:10A55000022A49D14A68507811780002244A0843F7
:10A560008018042840D801F07BF803121D1B23003B
:10A57000F06801F0DDF8021CC0B2B84200D93A1C04
:10A58000D2B22000F1682A8000F09AFF06E0022291
:10A59000F3681B882A8023701B0A63700020F8BDB3
:10A5A0000622EEE701232B80F3681B782370F5E782
:10A5B000F368002B16D008222A801A8822701A8885
:10A5C000120A62705A88A2705A88120AE2709A8837
:10A5D00022719A88120A6271DA88A271DB881B0ADA
:10A5E000E371DBE72B80D9E701202B80D7E7C0465A
:10A5F00000D6FFFFF7B516000A781D0008AB1F88CC
:10A600000C000123022A18D14A6850781178000200
:10A610002B4A0843801803280FD801F021F802259F
:10A620004439E06801F084F8C0B20723B84204D38B
:10A630007B190193152B02DD0D231800FEBDE06888
:10A640002A003100C01900F03BFF6B4600209B88B8
:10A65000E268D0541B4B1B68834203D01B688342C3
:10A6600000D098470023E8E70B23002FE5D1022D07
:10A67000E2D1737832781B021343E2681380114BE6
:10A680001B68002BEED01B68002BEBD00120E8E705
:10A690000B23002FD1D1062DCED12A003100E06846
:10A6A00000F00EFFDEE70B23002FC6D1012DC3D132
:10A6B00032787533012AC0D8E3681A70D2E7C046F1
:10A6C00000D6FFFF4868FF1F70B50C001500072873
:10A6D00037D800F0C5FF041436361B36242E182058
:10A6E00015290BD8184E16220021300000F010FF5B
:10A6F00022002900300000F0E3FE002070BD182089
:10A700000229FBD11288114B1A80F6E7182008297C
:10A71000F4D10A000E48290001F07AF8EDE718207C
:10A720000129EBD10B4B10780B49DA69FFF7DEFEFC
:10A73000E3E718200129E1D1064B10780749DA6BCD
:10A74000F4E70220DAE7C0463068FF1FD643FF1F58
:10A75000CC43FF1F5C43FF1F8443FF1FA443FF1F25
:10A76000030010B50020DB0704D50721024A034887
:10A7700000F08CF810BDC0468CBD00115C43FF1F7B
:10A78000054A03001068002803D082889A4201D14C
:10A79000806870470068F6E7406AFF1F0A88030078
:10A7A00008009A4204D08A8804309A4200D00020DF
:10A7B00070470000F8B5F22200230D4F0D4E796866
:10A7C000050042433370994200D07B600A4C00215F
:10A7D000200000F09DFE00231A007C60AB4202D1F5
:10A7E00000203370F8BD01332280DBB2F234F5E78C
:10A7F000386BFF1F366BFF1F446AFF1F73B56B4634
:10A8000001900600684615001980FCF74DFF041EF4
:10A8100011D1002D0FD07689002E11D00C2001F01F
:10A8200027F800280ED0084A0460136886808560E7
:10A83000002B02D11060200076BD1A001B68F7E7DC
:10A840000224F8E71324F6E7406AFF1F01210022E3
:10A850000A4B10B549420A4C198099809A719A7036
:10A86000084B2070012019805A60FFF7A3FF207861
:10A87000FCF778FF0448FDF733FF10BD5068FF1F59
:10A88000406BFF1F386BFF1F39A90011022310B561
:10A89000002802D0FFF7B2FF0300180010BD00002F
:10A8A000030010B50020DB0704D50421024A034849
:10A8B000FFF7A4FF10BDC046A0BD0011DC43FF1F81
:10A8C000F0B50E2687B003930CAB1F8802ABF618C9
:10A8D0000500080031000292FDF768F8040001202D
:10A8E000002C0FD03088FFF74BFF03000E20002B09
:10A8F00008D05E68002E05D021002800039B029A34
:10A900000097B04707B0F0BD0A4B10B5984207D189
:10A910000122002352420A808B708A808B7110BD05
:10A92000FFF73CFF0028FAD001235B42038000239D
:10A930008370F4E7FFFF0000F8B5050001290AD194
:10A94000134E00243388F227AB4219D02800114956
:10A95000FFF7DAFF06E0022904D10139FDF73EFFD7
:10A960000028EDD0F8BD3B0063437268D018D35A7D
:10A97000002B09D03A00002100F0CAFD0134E4B2F6
:10A98000054B1B78A342EED801235B423380DDE701
:10A99000386BFF1F5068FF1F366BFF1F10B5FFF7A6
:10A9A000FDFE03000020834200D0987810BD000017
:10A9B000F0B589B01C000EAB80CB03901E8810ABA5
:10A9C0001B78049202930B7A0D00DB0616D42B78C9
:10A9D0000593022B24D00498FFF7D2FE002812D052
:10A9E00003689C46002B0ED0029B22000193290095
:10A9F0003B00644603980096A04705E00498FFF7E3
:10AA0000BFFE002802D10E2009B0F0BD8368002BE4
:10AA1000F9D00A222900039898470028D7D0F3E7F5
:10AA20006B6858781A786B4B000210439842D2D862
:10AA3000043B984210D2684B984242D015D8674BDD
:10AA4000C0180128C7D80B20002EDDD1EB681A787A
:10AA500059683A80200028E0614BC018032800D9CB
:10AA600079E000F0FDFD846A789E5E4B9842B2D199
:10AA70000B20002EC8D101233B80EB6831001B78EE
:10AA800023706889013080B2FCF790FF3A88031E7A
:10AA90000ED0017802328A183A8042896270428967
:10AAA000120AA27059680278E01C00F009FD06E065
:10AAB00004323A8031000422601C00F029FD00209D
:10AAC000A2E70B20002E9FD1EB6807A91E88042364
:10AAD0003B80330A300026706370FCF767FF051E69
:10AAE00028D004AB9A890E2304A95B183E49C66896
:10AAF000FCF7D0FF00280BD12B783C486A680599F9
:10AB0000FBF786FB002803D1012304AA5B42D38113
:10AB10003278022A06D17168201D00F0D1FC3B88F2
:10AB200002333B800E2304AA9B181B88A3701B0AC8
:10AB3000E370C4E704ABDE81F4E70B20002E00D005
:10AB400062E7E9680398FFF729FF02233B80207042
:10AB5000000A6070B3E70B20002E00D054E70222F9
:10AB6000EB681B883A8023701B0A6370A7E7E868CC
:10AB700000F0DEFDC2B203000720B24200D243E77C
:10AB80000DD00299DBB27118994202DB921BD3B24D
:10AB90000293029BE9681A003B8089195AE7002357
:10ABA000F6E70B20002E00D02EE70722EB683A8054
:10ABB0001A7822705A7862705A88A2705A88120ADB
:10ABC000E2701A792271DA886271DB881B0AA3713C
:10ABD00075E7C046042900000228000000D8FFFFE6
:10ABE000FFD6FFFF03280000FFFF0000D0BC0011CC
:10ABF000F0B58DB06B460020089120229B5E834209
:10AC00003DDAA64B187800F09BFE071E32D0037881
:10AC1000B02B2CD10079023816281FD800F0D0FCB8
:10AC200017001E001E001E0031001E0096001E00B0
:10AC30001D011E0052011E0073011E00CD011E00E9
:10AC400050021E001E001E008E021E00E302944BE6
:10AC500094491B8878880B80FBF71AF83800FCF7BA
:10AC60009BFF914B1B68002B01D0380098473800A0
:10AC700000F006FE8020089B0002434018000DB043
:10AC8000F0BDEE220021874800F042FC0BAA3B7B7E
:10AC90007989388900923A000D32FCF79FFD040053
:10ACA000804B1B78002C3FD146E0804B7888059381
:10ACB0007F4B4100CB5A0BAE073BDBB2328802938D
:10ACC000002301937B4B210006930093059BFFF724
:10ACD0006FFE744D002810D1069B3A8A1B889A4259
:10ACE0000BD138000599123000F082FC002804D006
:10ACF0002B7862899B00EB185A80162306A81B1834
:10AD0000328820007989FCF7C5FE2B7804009A0070
:10AD1000AA1851880029C3D00133DBB22B70002858
:10AD200007D006A9C98A9180634A12889A42BCD882
:10AD300002E0012149429180002B04D059497888D2
:10AD4000FAF7DAFF8AE73E890A2479E000253E898E
:10AD5000574B06937B88069A5B009B5A033B9D42A8
:10AD600002DB002DF0D05BE0162206A812183B7B18
:10AD7000798900923A0030000D32FCF72FFD0590E2
:10AD8000002858D04689017A7888FCF7F1FC041E27
:10AD900044D1464B78880793069B4100C95A454BDE
:10ADA0000439C9B206AAD28A06930291019400938B
:10ADB0000599079BFFF7FCFD041E2FD1069B39491F
:10ADC0001A88931C002D26D14B807988384B490076
:10ADD000CB5A5119033B8B4220DD059B31485B89DF
:10ADE00041190B71A91C0135C9B2EDB20591451984
:10ADF0001B0A2B71059B2D490433181800F060FBCA
:10AE00002C4B059A1B88D318DDB22C4B9E4205D0E3
:10AE10000136B6B29CE749889942D6D0002D0CD0B5
:10AE2000204C2800618800F003FD20702100788804
:10AE3000FAF772FF12E7059CF0E7002C00D183E7D8
:10AE40007B78142B00D109E716493B794E800B70B3
:10AE50000C717888FAF712FF00E7162406ABE418A5
:10AE600021003889FCF7A2FD011E00D1B7E17888E6
:10AE700022880F4C45002C5B0A4D013CE4B2029441
:10AE800000240F4B01940095FFF792FD041E00D0A3
:10AE900014E129007888FAF74FFFDFE6406BFF1FC7
:10AEA000C842FF1F5868FF1F4C68FF1F4C69FF1FF7
:10AEB0008864FF1F3C6AFF1FC642FF1FFFFF0000A0
:10AEC0005A68FF1F162406ABE41821003889FCF7E6
:10AED0006DFD011E00D182E178882288AE4C4500CC
:10AEE0002C5BAE4D013CE4B202947C89AC4B0194E6
:10AEF0000095FFF75DFD041E00D0DFE02900788893
:10AF0000FAF724FFAAE60025A44B1D803B00F63388
:10AF10001B78A24A78880792AB4208D99E4B1288C8
:10AF20000693069943005B5A013B9A4203DB07995B
:10AF3000FAF716FF92E616246B00FB18059306AB92
:10AF4000E418059B21001889FCF730FD011E03D190
:10AF5000059B01241E8973E77888924B2288069C02
:10AF6000099343001B5B904E013BDBB2029300232D
:10AF700000960193099BFFF71BFD041E02D0059B61
:10AF80001E895DE77B88069A5B009B5A079A1088AA
:10AF900032881218934202DC1B1A013B33807F4C2B
:10AFA000023032880999001900F08AFA2388328821
:10AFB00001359B182380EDB2A8E70BAA3B7B79896A
:10AFC000388900923A000D32FCF708FC0025059004
:10AFD000059B002B04D10A24002D00D16EE060E017
:10AFE000059B7888197AFCF7C3FB0100041E63D126
:10AFF000694C6C4B788806940993069B4400E45A8C
:10B00000694B063CE4B20BAE32880793029401917F
:10B0100000930599099BFFF7CBFC041E4CD1079BBD
:10B020005E491B881A1D002D30D14A80059B5B4C60
:10B030005A8963191A716B1C9BB2E318120A1A71B0
:10B04000162306A832881B1879890598FCF722FD7B
:10B05000FF21AA1C2E1D03350B00059092B2B6B23B
:10B06000ADB2002803D006ABDB8AD9B21B0AA21806
:10B07000651911712B714C4D301D2A8849492018D2
:10B0800000F01EFA2B88F618B5B2A1E74988914264
:10B0900007D17A8806995200525AEB18053A9A421B
:10B0A000C4DC3E4C2800618800F0AAFB207021001F
:10B0B0007888FAF75FFED1E5002DF2D13E89BFE630
:10B0C000162606ABF61831003889FCF76FFC3D00F8
:10B0D0000400FA3500282DD0037A9B060CD40022F8
:10B0E0007B893989788800923A000C32FFF7E8FBB7
:10B0F000041E10D03E8915E03088FFF741FB002880
:10B100001AD08368002B17D0210012227888984724
:10B11000041EE4D0EEE72B78002B02D17888FAF7F2
:10B1200039FE00262B78002B00D097E5002C00D1AB
:10B1300094E585E60124DDE70E24DBE7162506AB62
:10B14000ED1829003889FCF731FC041E47D0037A3A
:10B150009B0611D4154A7B881188994203D0144864
:10B16000814207D11380134BF2261D780023D9B2F8
:10B17000A94221D30924A1E72888FFF701FB002871
:10B180002FD08368002B2CD021001222788898477A
:10B19000041EDFD092E7C0468864FF1F5868FF1F77
:10B1A0005A68FF1F4C69FF1F3C6AFF1F386BFF1F67
:10B1B000FFFF0000366BFF1F310059435468013315
:10B1C0006018615A0029D2D13C0008342100F222D3
:10B1D00000F076F921007888FAF7E4FD3EE50124D5
:10B1E0006CE70E246AE71D4B1A887B889A4231D09F
:10B1F0007888FAF7E1FD31E5F22305985168434379
:10B20000CD18C95A00291FD03B7A012B0BD16C886D
:10B21000AB887888AA1D0094FFF752FB041E02D069
:10B2200000233B722E88F2220021280000F070F9E2
:10B2300000232B80059B0133DBB20593084B059956
:10B240001B78064A8B42D7D801235B421380002C1F
:10B25000CED0F5E5002634000596EFE7386BFF1FEA
:10B26000366BFF1F70B504000E001500FFF796FA4D
:10B27000031E08D131000548FFF790FA03001120A2
:10B28000002B02D01C8000209D7070BDFFFF0000CD
:10B29000F8B50B4F06003B780D001400FF2B0ED0C5
:10B2A0000A2000F01DFB011E09D0B12303800023FA
:10B2B00046800371C5800481387800F0F1FAF8BD4A
:10B2C0001D44FF1FF7B50F0008A90600088809A94B
:10B2D0000B240988002821D10234022B1ED1557875
:10B2E00013782D021D432B008B4301937334002BE5
:10B2F00014D1FB68300019000093FFF74FFB019C4D
:10B3000085420BD02A0030000099FFF7ABFF041EE6
:10B3100004D12A0030007989FFF7BAFF2000FEBD72
:10B32000F0B50E7885B003900AA805880120022E9A
:10B330000DD14C682778647824023C43054FBC4209
:10B3400005D10398DBB201960095FFF7BBFF05B06E
:10B35000F0BDC04602290000034B10B51B68002B4E
:10B3600000D09847FEE7C046446BFF1F07B501A811
:10B37000FFF7F2FF044A05480021121A00F070F8A6
:10B38000F8F7C0F9FEE7C046486BFF1F2044FF1FD7
:10B3900001B40248844601BC604700BF753AFF1FF4
:10B3A00001B40248844601BC604700BFB54C0100AF
:10B3B00001B40248844601BC604700BF1147010048
:10B3C00001B40248844601BC604700BF5D1700001D
:10B3D00001B40248844601BC604700BF4938FF1FE2
:10B3E00001B40248844601BC604700BF3119FF1F09
:10B3F00001B40248844601BC604700BF5139FF1FB9
:10B4000001B40248844601BC604700BF014C010002
:10B4100001B40248844601BC604700BFC94A01002C
:10B4200001B40248844601BC604700BF893BFF1F4E
:10B4300001B40248844601BC604700BFA136FF1F2B
:10B4400001B40248844601BC604700BFC536FF1FF7
:10B4500001B40248844601BC604700BF0D31FF1FA4
:10B4600001B40248844601BC604700BFB70E00002B
:10B4700001B40248844601BC604700BF2146010078
:10B4800001B40248844601BC604700BFC5210000EA
:10B4900001B40248844601BC604700BFA54F0100CB
:10B4A00001B40248844601BC604700BF012400008B
:10B4B00001B40248844601BC604700BF691F000018
:10B4C00001B40248844601BC604700BFE94C01005A
:10B4D00001B40248844601BC604700BFD532FF1F5B
:10B4E00001B40248844601BC604700BF453BFF1FD2
:10B4F00001B40248844601BC604700BF29510100E5
:10B5000001B40248844601BC604700BFD94901002C
:10B5100001B40248844601BC604700BF154D0100DC
:10B5200001B40248844601BC604700BF51250000B9
:10B5300001B40248844601BC604700BFE117000027
:10B5400001B40248844601BC604700BF456B01005E
:10B5500001B40248844601BC604700BFA94601000F
:10B5600001B40248844601BC604700BF091B0000CB
:10B5700001B40248844601BC604700BF6D30FF1F24
:10B5800001B40248844601BC604700BFEDA500003D
:10B5900001B40248844601BC604700BF311B000073
:10B5A00001B40248844601BC604700BF2D2EFF1F36
:10B5B00001B40248844601BC604700BF017F00001F
:10B5C00001B40248844601BC604700BF9D3BFF1F99
:10B5D00001B40248844601BC604700BF090E000068
:10B5E00001B40248844601BC604700BF8D120000D0
:10B5F00001B40248844601BC604700BFCD4C010045
:10B6000001B40248844601BC604700BF093AFF1FED
:10B6100001B40248844601BC604700BF8939FF1F5E
:10B6200001B40248844601BC604700BF6DBC000005
:10B6300001B40248844601BC604700BF055E0000BB
:10B6400001B40248844601BC604700BF3D180000B9
:10B6500001B40248844601BC604700BFF30E0000FD
:10B6600001B40248844601BC604700BF753BFF1F20
:10B6700001B40248844601BC604700BF0D5201007E
:10B6800001B40248844601BC604700BF3520FF1F5B
:10B6900001B40248844601BC604700BFAD32FF1FC1
:10B6A00001B40248844601BC604700BF9537FF1FC4
:10B6B00001B40248844601BC604700BF8B520100C0
:10B6C00001B40248844601BC604700BFC92600009F
:10B6D00001B40248844601BC604700BF79180000ED
:10B6E00001B40248844601BC604700BF9536FF1F85
:10B6F00001B40248844601BC604700BFED4A010026
:10B7000001B40248844601BC604700BF8552010075
:10B7100001B40248844601BC604700BF75A900001F
:10B7200001B40248844601BC604700BF056A0000BE
:10B7300001B40248844601BC604700BFDD520100ED
:10B7400001B40248844601BC604700BFDD660100C9
:10B7500001B40248844601BC604700BF3555000073
:10B7600001B40248844601BC604700BF3533FF1F67
:10B7700001B40248844601BC604700BF554901003E
:10B7800001B40248844601BC604700BF2526000082
:10B7900001B40248844601BC604700BFC9A900004B
:10B7A00001B40248844601BC604700BF613BFF1FF3
:10B7B00001B40248844601BC604700BF5D34FF1FEE
:10B7C00001B40248844601BC604700BF8530FF1FBA
:10B7D00001B40248844601BC604700BF5522000006
:10B7E00001B40248844601BC604700BFE92800005C
:10B7F00001B40248844601BC604700BF8D1BFF1F97
:10B8000001B40248844601BC604700BF090E000035
:10B8100001B40248844601BC604700BF810E0000AD
:10B8200001B40248844601BC604700BFF13AFF1FE3
:10B8300001B40248844601BC604700BF350E0000D9
:10B8400001B40248844601BC604700BF5147010073
:10B8500001B40248844601BC604700BF21240000B7
:10B8600001B40248844601BC604700BFB14E0000ED
:10B8700001B40248844601BC604700BF3D4B010053
:10B8800001B40248844601BC604700BF434D01003B
:10B8900001B40248844601BC604700BFB3520100B6
:10B8A00001B40248844601BC604700BF594F010003
:10B8B00001B40248844601BC604700BF851F0000F8
:10B8C00001B40248844601BC604700BFC939FF1F6C
:10B8D00001B40248844601BC604700BF59520100D0
:10B8E00001B40248844601BC604700BF1D4D010001
:10B8F00001B40248844601BC604700BFC530FF1F49
:10B9000001B40248844601BC604700BF156B0100CA
:10B9100001B40248844601BC604700BFE54800000E
:10B9200001B40248844601BC604700BF1D3BFF1FB5
:10B9300001B40248844601BC604700BF4550000086
:10B9400001B40248844601BC604700BFF54E0100C7
:10B9500001B40248844601BC604700BFC51D000019
:10B9600001B40248844601BC604700BFADAE000090
:10B9700001B40248844601BC604700BF4D1F00006F
:10B9800001B40248844601BC604700BFF94C010085
:10B9900001B40248844601BC604700BF0519FF1F7F
:10B9A00001B40248844601BC604700BF291C000066
:10B9B00001B40248844601BC604700BF3D39FF1F07
:10B9C00001B40248844601BC604700BF1D4B010022
:10B9D00001B40248844601BC604700BFD91B000087
:10B9E00001B40248844601BC604700BF6571010094
:10B9F00001B40248844601BC604700BFC56D010028
:10BA000001B40248844601BC604700BF45510100B3
:10BA100002000300040305030603070208030903E9
:10BA20000C030D001600090100000000E93A0011A6
:10BA30001D3B0011000000000200000042BA00118E
:10BA4000192A0F181EFF4C0012190A00F1590000A4
:10BA5000FD24000041460100E97D0011FD9D00111B
:10BA600051720011ED7B001181530011F1AB0011F7
:10BA7000354F00112940001159410011000000000C
:10BA8000161600000200000090BA0011F4FFF3FF48
:10BA9000D2FC0000994200110000000000000000EC
:10BAA0004449590042322E3000303032300067694C
:10BAB000746875622E636F6D2F70767678004B45D3
:10BAC0005900000002000000D8BA0011292A282AD3
:10BAD000272A262A252A242A0A1800000500000001
:10BAE0001F501D10023CB400000120002000000087
:10BAF000090060003031323334353637383941424D
:10BB0000434445460000000001A000000000000082
:10BB10006410B71DC8206E3BAC30D9269041DC764E
:10BB2000F4516B6B5861B24D3C7105502083B8EDF8
:10BB300044930FF0E8A3D6D68CB361CBB0C2649B1C
:10BB4000D4D2D38678E20AA01CF2BDBDDC1D2F1C26
:10BB50009A1A1C19B3175E161D15EE13C1122B127B
:10BB6000C210D10FEE0E170E4D0D8E0CD902D2025F
:10BB7000DA02D202D902D202D702D202D902D2020A
:10BB8000DA02D202C002D202DA02D202D902D20210
:10BB9000D502D202D902D202D702D202C002C0021A
:10BBA000C502C204FF02FF04FF1ED604D604D2045D
:10BBB000EB04FF04EB04FF04D404FF04D404FF04EB
:10BBC000D404D808D904DB04D904D904D904D40492
:10BBD000FF04D204FF04D604FF04D604FF04D604F5
:10BBE000D408D604D404D608D204EB04FF04EB0432
:10BBF000FF04D404FF04D404FF04D404D808D904F7
:10BC0000DB04D90CD404FF04D204FF04D604FF04DF
:10BC1000D604FF04D604D408D604D404D608D2042B
:10BC2000EB04FF04EB04FF04D404FF04D404FF047A
:10BC3000D404D808D904DB04D90CD404FF04D204FA
:10BC4000FF04D604FF04D604FF04D604D408D604A7
:10BC5000D404FF1EFB349B5F8000008000100000B6
:10BC600000000000535E0011DD740011775E0011CA
:10BC7000E5780011FB5E0011BB780011715F0011C7
:10BC800091780011C35F0011597A00112B600011E7
:10BC9000597A00115D600011137A0011715F001173
:10BCA00049780011E95F0011F179001100000000EE
:10BCB00000000000CF600011F17900113161001126
:10BCC000F5740011052A042A012A002A02290328F2
:10BCD00001280028011800180000000000000000E2
:10BCE00000000000000000870101020102010102C2
:10BCF0000102030304010301010101010303020125
:10BD000003000D000E0010001100130014010701C4
:10BD100008010A010B011C011D02040205020702B1
:10BD2000080219021A021C021D0301030203170074
:10BD30000201000504000807000B0A001716001D89
:10BD40001C010201010504010E0D01111001141363
:10BD5000011716011A19020201020B0A020E0D0246
:10BD60001110021413021716030504030807030B2E
:10BD70000A030E0D0001020307090A0B0E0F101132
:10BD800012141718191A1B1F2021220039A500119F
:10BD9000F5A500110000000002000000D6BC001153
:10BDA0000000000021B300110000000002000000AC
:04BDB000D4BC0011EE
:020000041FFFDC
:1000000000000000913F00114CBA00114ABA0011E3
:10001000A861FF1F000000000000000000000000B9
:1000200000000000000000000000000000000000D0
:1000300000000000000000000000000000000000C0
:1000400000000000000000000000000000000000B0
:1000500000000000000000000000000000000000A0
:100060000000000000000000000000000000000090
:100070000000000000000000000000000000000080
:100080000000000000000000000000000000000070
:100090000000000000000000000000000000000060
:1000A0000000000000000000000000000000000050
:1000B0000000000000000000000000000000000040
:1000C0000000000000000000000000000000000030
:1000D0000000000000000000000000000000000020
:1000E0000000000000000000000000000000000010
:1000F0000000000000000000000000000000000000
:1001000000000000000000000000000000000000EF
:1001100000000000000000000000000000000000DF
:1001200000000000000000000000000000000000CF
:1001300000000000000000000000000000000000BF
:1001400000000000000000000000000000000000AF
:10015000000000000000000000000000000000009F
:10016000000000000000000000000000000000008F
:10017000000000000000000000000000000000007F
:10018000000000000000000000000000000000006F
:10019000F932FF1F5931FF1FC16601000000000046
:1001A000000000000000000000000000000000004F
:1001B000000000000000000000000000000000003F
:1001C000000000000000000000000000000000002F
:1001D000000000000000000000000000000000001F
:1001E000000000000000000000000000000000000F
:1001F00000000000000000000000000000000000FF
:1002000000000000000000000000000000000000EE
:1002100000000000000000000000000000000000DE
:1002200000000000000000000000000000000000CE
:1002300000000000000000000000000000000000BE
:1002400000000000000000000000000000000000AE
:10025000000000000000000000000000000000009E
:10026000000000000000000000000000000000008E
:10027000000000000000000000000000000000007E
:10028000000000000000000000000000000000006E
:10029000000000000000000000000000000000005E
:1002A000000000000000000000000000000000004E
:1002B000000000000000000000000000000000003E
:1002C000000000000000000000000000000000002E
:1002D000000000000000000000000000000000001E
:1002E000000000000000000000000000000000000E
:1002F00000000000000000000000000000000000FE
:1003000000000000000000000000000000000000ED
:1003100000000000000000000000000000000000DD
:1003200000000000000000000000000000000000CD
:1003300000000000000000000000000000000000BD
:1003400000000000000000000000000000000000AD
:10035000000000000000000000000000000000009D
:10036000000000000000000000000000000000008D
:100370006DB300110000000000000000000000004C
:10038000000000000000000000000000000000006D
:10039000000000000000000000000000000000005D
:1003A0000000000000000000000000000D1BFF1F07
:1003B000000000000000000000000000000000003D
:1003C000000000000000000000000000000000002D
:1003D000000000000000000000000000000000001D
:1003E000000000000000000000000000000000000D
:1003F00000000000000000000000000000000000FD
:08183800506FFF1F4118FF1F54
:10184000024981F3088802F033FC0000506FFF1F4B
:1018500070B500241E491F4A1F484C6308CA1B0567
:101860001B0DE4188242F9D11C4B80228B630021AE
:1018700009201B4B920519621A4B1B4DDA671B4B53
:10188000DA688243DA609A68194802409A60112047
:10189000296002F0B9F8112002F096F880226B6CF2
:1018A000112093436B64EE23DB006343114A1B0C4E
:1018B00013840122104B9A7401F004FC0F4B1B7827
:1018C000002B04D10E4B1021187802F091FA70BD54
:1018D000000005408805054000060540FF010000A6
:1018E00000F0004004E100E0003800403CF000401F
:1018F000FFDFFFFF2061FF1F1462FF1F4A64FF1F0D
:101900004862FF1F10B502F083FB072804D012289D
:1019100008D0022808D010BD044A0420136B0133FC
:101920001363F8E70220F6E71420F4E73065FF1FA1
:10193000F8B507000C0026002500503630785135E8
:10194000002804D10300287058342370F8BD29788A
:10195000CA00481E8141A3183800A25C5B68C9B266
:10196000FFF7D0FF00280DD12B78DA00A218013341
:1019700050602B703378044A013B3370136A013393
:101980001362D8E70123DFE73065FF1F5C23434381
:10199000074910B5C9180B0058331B78012B05D126
:1019A000FFF7C6FF034A936A0133936210BDC04636
:1019B0006465FF1F3065FF1F10B502F0F1FA064A9B
:1019C0000121130010CB4942D967044B136002F088
:1019D00087FA200010BDC04600E100E010001000B2
:1019E00010B5040002F0DCFA024B1C6002F078FA39
:1019F00010BDC04600E100E0431E5A425341A02200
:101A0000F0B5D2015B421340154D164A40019B18B8
:101A10002A18127E8BB00191002A1BD01A000832BE
:101A2000D46F0022E6B206AFE4B294420EDC28186E
:101A3000C369002B08D0019902AA117106AA049269
:101A400002AA167303A898470BB0F0BD1978B954D1
:101A50000132EAE71A7D1A7806AB01261A70E6E72A
:101A6000F067FF1F00400040F0B5254B0400400127
:101A7000C25C85B0002A2BD01A18117E002927D00D
:101A8000917E002924D01179022921D11689D78885
:101A9000D168F51BADB22A1C102D00D9102292B2CC
:101AA000BE4217D11818012303710023C269C380F5
:101AB00003819A4206D068460321037301710293A1
:101AC00001A890470820002C00D0192001F0FAFA54
:101AD00005B0F0BD013C65426C41A0256442ED01BA
:101AE0002C40084D1B186419074D0633013A92B279
:101AF000AA42EDD01888461C1E80085C2070F5E7CD
:101B0000F067FF1F00400040FFFF00000F220E4B58
:101B100010B59868104002380A280BD802F02AF84D
:101B20000D0A0B0A0A110A0A0A0A060002210020FD
:101B3000FFF762FF10BD0121F9E70020FFF794FFD6
:101B4000F8E7DB6FF6E7C046004000400F220E4B7F
:101B500010B59868104002380A280BD802F00AF82D
:101B60000E0A0B0A0A120A0A0A0A060002210120BA
:101B7000FFF742FF10BD01210800F9E70120FFF740
:101B800073FFF7E7DB6FF5E70090004013B5334CC8
:101B90002378072B3DD8324B1A78324B002A39D1A3
:101BA0008022196852020A431A60252001F0ECFED7
:101BB00020232D4A11680B43802113606B460422B9
:101BC000C90508680733104228D080210422C905BE
:101BD000C86810422ED080212020C905CA688243DF
:101BE000CA6014221A701A78002A2FD18021C905E0
:101BF000C86820320243CA6014221A701A78002A78
:101C000028D11A4B1A7D22785A601D221A70593237
:101C1000DA6013BD1A6816490A40C5E7086802432E
:101C20000A6014221A701A78002ACED01A78013A63
:101C3000D2B2F7E7C8680243CA6014221A70197852
:101C40004A1ED2B21A700029F9D1C4E71A78013AB3
:101C5000D2B2C7E71A78013AD2B2CEE75843FF1F93
:101C60002044FF1F3CF000405043FF1F0020004075
:101C7000FFFFFEFF564B70B51B68012B03D1554A81
:101C8000936D0133936501F0A3FF534B534A1860E2
:101C9000534B544C1A600123534A1360534A136048
:101CA0002378002B06D006225149524802F0C8F88A
:101CB00000232370504A514B10681B78C1B2002B8F
:101CC0000ED14F4CC0B223785BB2002B4FDB237890
:101CD00024785BB264B21B0424021B191B18136026
:101CE0000B1C50294ED95023464A47491078DBB285
:101CF000FF2202284BD10868444C454D267890437A
:101D00002A78964254D9227824782E78023B5D10A6
:101D1000A31B6B435201D31A10335B1118430860A5
:101D200002F02EF8031F012B45D83A4B1B78002BED
:101D300006D0394B1B78002B02D0002002F018F996
:101D4000A122364B92009978354B4A431B689B1869
:101D5000832292009B181B78033B012B03D8AF20F2
:101D6000400002F0A5F801222E4BDA8270BD2378E4
:101D700024785BB264B2FF33FF341B0424021B19C6
:101D80000138ABE7CAB2022AAED20223ACE7086838
:101D9000254C264D267890432A78964208D92278F9
:101DA00024782D78023B5B10641B63435201B2E739
:101DB0002378DBB2B2E70228D5D11D4B1B78013B5B
:101DC000022B03D91B4B1B78022BCCD16C20C8E70C
:101DD0009809FF1FFC0FFF1F7C64FF1FFF3F0000DF
:101DE000141003408064FF1F0C10034000100340D8
:101DF000D50BFF1F7211FF1FB40003408C09FF1F9A
:101E0000680AFF1F490AFF1F94000340460AFF1F8C
:101E1000470AFF1FF908FF1F2209FF1F300DFF1F90
:101E20003409FF1FBC0BFF1F440AFF1F450AFF1F99
:101E30001C09FF1F2309FF1F10B501F0C9FF002275
:101E4000014B1A8010BDC0467864FF1F10B502F028
:101E5000BFF8A121054A89009478054A61431268B8
:101E6000044B5218528C1A8010BDC046300DFF1F13
:101E70003409FF1F7864FF1F10B50D4B0D4A997888
:101E8000A1239B004B431268D218531DD97F0A4BE4
:101E90001B88994209D2441C07D0C82805D0D269B2
:101EA0005B1A5A43054B5343C01801F0E9FF10BDBC
:101EB000300DFF1F3409FF1F7864FF1F71020000FF
:101EC00070B5244D2B68002B28D001F0A9FF2B689A
:101ED000D8402B680400002B27D002F091F82B6823
:101EE000D8401D4B1D4A9978A1239B004B43126893
:101EF000D118D25C91239B00002A20D0CA5801320D
:101F0000CA50174B17491B680868834214D3D23B49
:101F1000181A012A1AD0144B186070BD01F080FF06
:101F2000124B196801F074FED3E702F069F80F4B09
:101F3000196801F06DFED4E70D495B18E8E7CA5057
:101F40000C4B1B68DB68E418201AE4E7F530FF301F
:101F5000E1E7C0461C08FF1F300DFF1F3409FF1FBB
:101F60009C09FF1F7C64FF1FA009FF1F1808FF1FAB
:101F70002DFF3F008464FF1F70B504000D00282969
:101F800016D10300A433C2881B889B1A0B4A9BB24C
:101F900093420DD906006A3605223100653001F002
:101FA0001FFE002804D13100200001F071FF70BD38
:101FB0002900200002F08CF8F9E7C046FE7F0000FF
:101FC000F8B50500012002F04BF8134CA36AA26A91
:101FD0009342FBD1114E336001F0F2FE1049030031
:101FE00008601048426894460F4A17680022BC45B2
:101FF00001D24268BA1A0D4802603268AD18A422B4
:10200000E562606A520302436262094A1278002A5A
:1020100001D00F3B0B60F8BD00F00040340AFF1FF9
:10202000E408FF1F28100040180AFF1F1C0AFF1FAA
:102030001C09FF1F70B580241025E405A3682B43FD
:10204000A36001F0E5FEA368AB43A36070BD000090
:10205000F7B5160080221C001023D205019191686B
:1020600005000B43936000225A4BD7301A6001F0F1
:102070006FFF9D232A002F009B00EB58CA320121DD
:102080000092FC37002B01D00021009A386801F043
:102090008FFE2900009BCB311A784F4BD3351A6045
:1020A0004B780A781B0213438A7812041A43CB78C0
:1020B0001B061343494A1BBA13604B790A791B026A
:1020C00013438A7912041A43CB7931001B06134358
:1020D000434A1BBA13606B782A781B021343AA7811
:1020E00012041A43EB781B0613433E4A1BBA1360D3
:1020F000019A330213433C4A13603C4B22001B1BE2
:102100009C4603293DDCB3089A0013005142B21AE1
:10211000032A46D1354AE018511A827840781204D1
:1021200000020243E05C043302430A600022FF2BFA
:102130004BDDF0222E4B12011A600F222D4B1A603C
:102140002D4A1368002BFCD00023224A2749136034
:10215000091B321D0B191B68043A180A23706070A2
:10216000180C1B0EA070E3700434002AF2DC8022ED
:1021700010213B68D20501333B6093688B43936029
:10218000F7BD6346D578981893782D061B042B432A
:10219000157804392B43557804322D022B43036004
:1021A000AFE7022A0AD1114AE05C511AE2185278CC
:1021B000120202430A6004339BB2B7E7012AB5D189
:1021C0000A4A521AE15C1160F5E7084959180A6099
:1021D0000433ACE7000004403C00044038000440F5
:1021E00034000440300004400C000440000104406E
:1021F000040004401000044014000440F7B515002A
:1022000080221C001023D2050091916807000B4327
:1022100093600023654AD730136001F099FE9D2337
:102220003E009B00F9583B00CA363200FC330029BF
:1022300000D07FE0586801F0BBFD390032785C4B7C
:10224000CB311A604B780A781B0213438A78AC466C
:1022500012041A43CB78281D1B061343554A1BBA98
:1022600013604B790A791B0213438A7912041A43CB
:10227000CB791B061343504A1BBA13604B7A0A7A78
:102280001B0213438A7A12041A43CB7A21001B06DD
:1022900013434A4A1BBA1360009A2B021343484A5D
:1022A00013602200474B1B1B0093009BCE785B18EA
:1022B00001938B7836061B0433430E78043833437E
:1022C0004E78043136023343019E33600328ECDC40
:1022D0000321A808431C9B002940800003292BD11F
:1022E0003849E5185E18A9786D78E35C09042D0279
:1022F000294319433160030008330021FF2B2DDDF2
:10230000314B324919600F21314B196001232749A4
:102310000B60304B19680029FCD006211B680B406C
:10232000042B20D080220020D20593680A318B43F1
:102330009360FEBD01217DE7022908D121495D1886
:10234000E1184978E35C090219432960D3E70129C0
:10235000D3D11C495918E35C0B60CCE71948181815
:1023600001600433CAE7002310490B606346002B69
:102370000CDC3B00FC335A68102101325A60802289
:10238000D205936801208B439360D2E7009B9B1892
:102390001B68190A13705170190C1B0ED37004239B
:1023A0005B4291709C440432E0E7C0460000044068
:1023B0003C00044038000440340004403000044035
:1023C0000C0004400001044004000440080F000019
:1023D000100004401400044070B5061E19D00222FB
:1023E0005A4B9B799343012B13D1594B1A78FF2AEF
:1023F0000FD15A78FF2A0CD19A78FF2A09D1DA78BE
:10240000FF2A06D11A79FF2A03D15B79FF2B00D16D
:1024100099E0504B0C201A78012A08D000224E4D2A
:102420001A7029780B00093B042B01D8212070BDBC
:102430004B1F012BFAD9454CA37B042B00D982E01A
:10244000A279032A00D97EE09A1ED2B2012A02D8CC
:1024500060881F2877D9002E56D0012E73D1A0880E
:102460000128E3D0002907D1581E032803D801F022
:1024700081FB121715122E702978481E032811D8D7
:102480000025364B1D602823237501F021FCA8424E
:1024900027D0A580CAE702212970EDE70421FBE7D8
:1024A0000321F9E707390129C0D82D490968C96A0C
:1024B0008906BBD52B4908780028B7D1012A01D954
:1024C000002BB3D102230B708021274D26338901C5
:1024D0002878237501F0A4FD80212878890101F076
:1024E00087FC0123A380214B1B78002B0AD0FA2202
:1024F00080211F4B92001B8809025A431A4B1878FF
:1025000001F096FB002092E701F04AFD2B78A680AF
:10251000073B012B03D917482E7001F091FB114B9B
:10252000114C1A78002A06D08021002220788901D7
:102530001A7001F075FD01F0D3FC802120780902AA
:1025400001F06EFDDEE7122071E7C046A60BFF1F0B
:102550006B09FF1F1A09FF1F1C09FF1F4809FF1FF6
:102560008464FF1F2309FF1F1B09FF1F2109FF1F91
:102570002C09FF1F0010004010B5002901D001F008
:1025800007FC10BDF7B5604B01919978A1239B0022
:102590004B435E4A060014681022E418D6235B0001
:1025A000E0583623FF33E35C00279343222B41D1CD
:1025B000574B0F3A1A600760012501F0C1FC019BDF
:1025C0001880E8235B00E35C002B01D0B34258DDA8
:1025D0000023504FFB70AD33FF33E3581A68002AD5
:1025E00003D09B88DB439B071DD03823FF33E35C7C
:1025F000002B18D09B235B00E35C002B13D1D1335D
:10260000FF33E35CB3420EDAA4235B00E15AE01827
:10261000090A023101F084FB23000122FE33013E4E
:1026200001351A87FA70E8235B00E35C002B2AD09F
:10263000A8B2FEBD03683D00002BBED081880430E7
:10264000090A023101F06CFBD6235B00E3581F60DE
:10265000B2E72300B133BA00FF33985801378188BD
:102660000430090A023101F05BFBE8235B00E35C04
:10267000BB42EEDCE822F61AED1800235200A35408
:10268000A6E70027F1E7200001F032FC00281FD068
:10269000002E1DDD7319882647190193B60020000E
:1026A00001F0A6FA5A308000201840680135818870
:1026B0000430090A023101F033FB200001F000FB75
:1026C000A3590133A351BD4202D0019B9D42E6D1E3
:1026D000114BE35C002BABD095239B00E35C002BFC
:1026E000A6D00E4BE15A0029A2D00D4AA35C994214
:1026F00002D90133A3549BE700231A212000A354DD
:1027000001F00EFC94E7C046300DFF1F3409FF1F97
:1027100000140340E010FF1F5A0200007202000084
:102720005E0200000D4970B54A6E0D4CD2038B69F4
:10273000D20BA24206D80B4D0224AA4204D901F0C2
:10274000E7FA70BD02246442E21815007E24254099
:102750002242F4D0A3432B438B61F0E700F000400A
:102760000A200000FC1C0000F8B51D4B1D4F1A7814
:10277000002A10D1BA7B002A02D101321A7003E07C
:10278000032AFAD0022AF8D001F0A2FA002201208E
:10279000154B1A70F8BD154B154D1C68154B9E78DE
:1027A00001232B702878C0B200F09EFBBB7B002B6E
:1027B0000BD101F0BDFAA1239B007343E4188323DE
:1027C0009B00E41823782B70E4E7032B02D101F07F
:1027D00067FAF0E70020022BDCD101F051FCEAE7B8
:1027E0001C09FF1FA60BFF1F2309FF1F3409FF1F32
:1027F000490AFF1F300DFF1FF0B587B00EAD2F78CF
:102800000FAD2D780593AC46634614000E4D0CAA0F
:1028100012782E7803930D9B009201932200059B62
:10282000029701F0A5FA2E70012C01D0042C08D1DA
:10283000802206498B889343054A1278D2011343BC
:102840008B8007B0F0BDC0461C09FF1F6C11FF1F35
:102850007809FF1F0B001B3B70B504003020E02BF4
:102860000DD81300E025493BFF3B9BB2ED00AB4286
:1028700005D8034B200019825A8201F071FA70BD0D
:102880008410FF1F10B501F0A3F9054B00205B6811
:10289000052B04D9034A5268D20200D4980810BD0F
:1028A00000100040FCE100E070B501F079FB0D4B39
:1028B0001B68FC33DC691D6AFFF7E4FF641984427E
:1028C00004D2094B01241B68002B07D004220024EA
:1028D000064B1A70064A93690133936101F000FBBD
:1028E000200070BD8464FF1F9809FF1F2309FF1F8C
:1028F000FC0FFF1F70B50C4D2B68FC335C6A01F0B8
:102900004FFBFFF7BFFF2B680025FC339B6AE318E2
:10291000834204D2054B1B68AB4200D1051B01F07A
:10292000DFFA280070BDC0468464FF1F9809FF1FAE
:10293000D722044B92009B5810B5002B00D098472B
:1029400010BDC0460000FF1F10B501F0FBF8FFF7F7
:10295000EFFF2749274BCA6D274C1A4084235B00A1
:102960001343CB65254B1B68186A01F079FB244B98
:10297000244A1A60244B254A1A60A022244B520094
:102980001A60244B187801F073F92000224901F0F5
:1029900077F90023A3600233A360204B2049236012
:1029A00003232048A36001F06BF910221E4BFF2087
:1029B0001A60802252031A60802292031A608022D9
:1029C00012041A6001F0D4FA012001F0C1F9FA20D2
:1029D000400001F0EDF8582001F06AFA134801F0C8
:1029E00067F9012001F084F9072001F0F9FA10BD20
:1029F00000F0004000FEFEFF141000408464FF1F42
:102A0000000003400180063DBC0003403408000084
:102A1000A40003404A0AFF1F71020000C30900001E
:102A2000FFFF3F002810004000E100E0307500008B
:102A3000674E336888331B6883F3088801F0C0F859
:102A4000644A6549136800200B401360634B644A75
:102A50001B68934200D1A6E001F032FB0221614ADB
:102A600013688B431360FFF76FFF5F4B5F4C187861
:102A7000C0B201F015FA0023A3600233A3605C4BDF
:102A80000120236001F0ECFA0323A36001F080FA37
:102A9000040001F09DF8050001F07AFA554B18602A
:102AA00001F016FA544B1968621A531EA14200D263
:102AB00013008022D203934201D39B029B0A326807
:102AC000D16AC90700D471E04C491C0C09689BB25B
:102AD0004C4359432402090A641803264849FC322E
:102AE00093680A6847489B1A474A0768126847492B
:102AF0009B18474A9A1833409208DB190A60036012
:102B0000042B03D9013233400A6003600E68414947
:102B1000A619300001F07CF83F4F3E493B68C318CE
:102B20003B603000019301F083F93C4E3068081897
:102B300038493060884205D9019B01333B6001F080
:102B400077F9316001F02CF9354B1B78002B0DD053
:102B500001F03EF8334B621B196812188A4232D2D8
:102B60004919091B091A304801F08AF82F4E337AA7
:102B7000002B0ED001F02CF8621BF1681218914264
:102B800024D94919091B091A294801F079F80023A9
:102B90003372284B83F3088801F07AFA002001F0A1
:102BA0008FFA01F03DF801F08BFA5CE7DC01990047
:102BB0000234641A5900641A09214B438033CB4014
:102BC000A408E41889E7FA218900CCE71A49DBE771
:102BD0008464FF1F1CF00040FFFFC1FF0C0AFF1FB1
:102BE000B641210310000040490AFF1F14100040A5
:102BF000C3090000100AFF1F340AFF1F380AFF1F15
:102C0000200AFF1F280AFF1F1C0AFF1F240AFF1F9C
:102C1000C4090000710200006008FF1F2C0AFF1F9A
:102C20001C09FF1FE408FF1F00100040740BFF1F6A
:102C30003C10004000000020DC050000A022054BF5
:102C400092009B5810B5002B01D0984710BD01F0A1
:102C500087F9FBE70000FF1FA122054B92009B585C
:102C600010B5002B01D0984710BD01F079F9FBE7B2
:102C70000000FF1FA222054B92009B5810B5002BAD
:102C800001D0984710BD01F06BF9FBE70000FF1F72
:102C9000A322054B92009B5810B5002B01D09847FA
:102CA00010BD01F05DF9FBE70000FF1FA422054BFA
:102CB00092009B5810B5002B01D0984710BD01F031
:102CC0004FF9FBE70000FF1F70B500F081FF4F4B8D
:102CD000186001F0BDF80400C30702D401F088F9C0
:102CE00070BD00224A4B1A604A4B187801380428FC
:102CF00029D800F03FFF0320181C2400200000F01A
:102D0000C7FF0128ECD0444C2378042B6ED101F08E
:102D1000F7F80028E4D001F033F9582001F0C8F8A2
:102D200002232370DCE7200000F09AFFE9E720008F
:102D300000F0E6FFE5E7200001F03AF9E1E72000C6
:102D400001F076F9DDE701F01BF80500012808D154
:102D5000324B1B78053B012B03D82000FFF76EFF99
:102D6000D1E72D4B1B78022B01D0052B20D1022D52
:102D700028D12B4B9B7BAB431CD12000FFF76CFF72
:102D8000264B18780128BED16405BCD424492522DD
:102D90004B7B034205D1233A13405A425341263319
:102DA0001A000B7D9342AED9322001F049F9AAE70F
:102DB000022D07D1194B1B78052B11D12000FFF7ED
:102DC00059FFDDE7012D0BD1012B03D12000FFF7C7
:102DD0005FFF98E7062B03D12000FFF767FF92E71C
:102DE000200001F0BDF8022D8DD1C9E7032B04D1DD
:102DF0000C4B987C01F054F972E7072B00D06FE779
:102E0000094B987B01F0DCF86AE7C0469C09FF1F7C
:102E10009809FF1F9009FF1F2309FF1F1C09FF1FAF
:102E2000A60BFF1FBC0BFF1FD40BFF1FFA210A4B81
:102E30000A4A49001A640A4A5A500A4A04395A503E
:102E4000094A08319A64094A5A50094A5C315A5071
:102E5000084ADA667047C0460000FF1FF927FF1FC7
:102E6000F528FF1FA928FF1FD923FF1F6927FF1F70
:102E7000791EFF1F4D1EFF1FF7B50B0CFF27012208
:102E8000009300233C001E001D009446019089B26F
:102E900062469A401000084018413618B6B2FF2F1B
:102EA00002D1012E00D19FB2009802401A41AD1804
:102EB000ADB2FF2C02D1012D00D19CB20133102BF9
:102EC000E6D10320012E07D1012D04D1019B24015D
:102ED000E4191C700138FEBD102EFCD10238102DF3
:102EE000F9D00230F7E700008023F7B59C46264B67
:102EF000264F01932649274A274D284C284B022864
:102F00001AD1604638600868264E30408026360365
:102F10003043086001990978002909D11660224AD6
:102F20002A60224A2260E02219689143A03A1BE0FD
:102F30008021C9021160F2E766463E600F68194EB3
:102F40003E408027FF023E430E6001990978002928
:102F50000DD1176001280ED1154A2A60154A22604A
:102F6000E02219689143C03A0A431A60F7BD8021F4
:102F700089021160EEE7E0210F4A02432A600F4AFE
:102F800022601A688A43F0E74B0AFF1FE000034003
:102F9000D80003409000034000000340500003406D
:102FA00040000340FFFFE3FF0280063D804508220A
:102FB0000180063D80660822008006988055082220
:102FC000F8B51E4B80261A680020140034403242A7
:102FD00032D11A681A4F32431A6001223B68063018
:102FE00093433B6001F03CF80122164D2B681E43D1
:102FF0002E603B680A2613433B608027BF00124BBC
:103000001B683B4211D1013EF6B2FF2E09D17E2250
:103010000E4B1C682B68E40B1440934323432B6036
:1030200005E0082001F01CF8E9E7002EEFD180222E
:103030002B68600893432B60F8BDC046C4F0004085
:103040005CF0004018F0004068F0004060F0004084
:1030500010B500F06DFF01215820034A00F030FF49
:10306000FFF7AEFF10BDC046600AFF1F10B5782203
:103070000021034800F0C4FD00F0FAFE002010BD5E
:103080007867FF1F70B5040000F08AFF00230C2052
:103090000B4A010059438D18515C00290DD0A14203
:1030A00008D1012300246B7000F0AAFE00F018FF85
:1030B000200070BD01330A2BEBD11224F6E7C04685
:1030C0007867FF1F70B5040000F06AFF0023190045
:1030D0001D000D4A1078002806D0A0420CD1557072
:1030E00001310C320A29F5D1002B0AD100F0C0FEC3
:1030F00000F0F6FE002070BD5078461EB0411B184F
:10310000EEE700F07DFEF3E77867FF1FF7B50400F8
:103110000C20002384460E4D019267465F43E85D14
:103120007E19A04212D000280BD10A4B9C46624661
:103130001B7808331370019B70707C557160B3600D
:10314000FEBD01330A2BE8D10320F9E70720F7E79A
:103150007867FF1F7467FF1F8020F8B5484BC005D4
:103160001B68C1248360474BFF251A680123134362
:103170004361454BA4001A68444B40211A60444BFC
:103180001A68444B1A60444B1A59AA431A51C52273
:1031900092009E58AE433143802699509F583F4934
:1031A000F6010F403E439E509E5880273602360A55
:1031B0003043985080201A5900020A4002431A51A5
:1031C00004341A59364E3F04324080263A431A518D
:1031D0001A5936061202120A32431A5108341A5981
:1031E00080260A4002431A51C32292009F58B446D7
:1031F000AF4337439F509F58294E0F4007439F507E
:103200009F58374080263604374380269F509F586A
:1032100036063F023F0A37439F50C0221F59AF4333
:103220003A431A511A591202120A1643C6221E5163
:1032300092009C58AC4365462C439C509C580025FA
:103240000C4020439850C72080001A58154C11405C
:10325000C02212020A431A50134B1B78DB08AB4200
:1032600001DC0020F8BD2378002B06D0A368002BDA
:1032700000D0984701350C34EEE71220F2E7C04643
:103280005443FF1F5043FF1FB0F000407067FF1F03
:10329000B4F000406C67FF1F00E100E0FF00FFFF9B
:1032A000FFFF00FF7867FF1F7467FF1F030010B563
:1032B0001F2809D8072200201340072404490A7850
:1032C000A24313430B7010BD00230620F5E7C04650
:1032D0007467FF1F054B06491B780A6805485B07A2
:1032E00002401B0B134300200B6070477467FF1FE5
:1032F0001CF00040FFFFC1FF70B50C25FFF7EAFF8F
:103300000A4B1C780A4BE4086543ED18002C01D1E8
:10331000200070BD2B78002B06D06B68002B00D0EE
:103320009847013C0C3DF1E71220F2E77467FF1F5C
:103330006C67FF1F70B50D00040000F031FE4021E6
:103340000F4AAD00136865198B431360AC4208D176
:10335000002202200B4B1A600B4B186000F0D8FDC6
:10336000FEE7637801212078002B00D0032100F0D4
:1033700037FD6178207800F0B3FC0434E6E7C046FE
:103380001CF00040C4F00040C0F000401FB5002118
:1033900002220B0001910091052000F069FE02233A
:1033A0000B490A681A42FCD120230393039B5A1E3F
:1033B0000392002BFAD1074A1368002BFCDA0B2486
:1033C0006C442000012100F043FE207804B010BDC1
:1033D00090C8004000C8004013B504000A4B019398
:1033E000019B002B01D1112016BDFFF7CFFF230059
:1033F0000340044205D0052000F032FE019B013B52
:10340000EDE71800F0E7C046FFFFFF0707B500F043
:10341000C7FD80220821D205936A0191002B01D1BA
:103420000739916202210C4A11600199481E0190EE
:103430000029FAD103311160053101910199481E2B
:1034400001900029FAD11160002B02D18022D2050F
:10345000936200F045FD07BD00C00040F0B52D4C63
:1034600089B02378002B4FD1FEF7A6FA02232A4F0A
:1034700003903A681A42FCD120230693069B5A1EF9
:103480000692002BFAD1254E3368002BFCDA01207E
:10349000FFF7A2FF011E02D0112009B0F0BD03000A
:1034A00003220190009005AD9F2000F0E1FD032173
:1034B000280000F0CDFD02233A681A42FCD12023F7
:1034C0000793079B5A1E0792002BFAD13368002BF3
:1034D000FCDA0120FFF780FF0028DDD10398FEF71A
:1034E0007FFAAA786B7811041B020B4329780B43EF
:1034F00063601300113B0A49052B07D80123934051
:10350000A3600B60012323700020C6E780231B0308
:10351000F6E7C0463C43FF1F90C8004000C800408B
:103520009808FF1F1E4B30B55A6818781D4B85B0A0
:10353000D31859424B4101210093002300F000FCB5
:10354000194B1A4A02259A6300221A6510325A65ED
:103550008022C4219D65164B1648D202DA67890085
:103560004258154B80241A4080231B0413434350B8
:10357000642341200393E40500F006FA402000F0A4
:1035800003FA6562039D6B1E0393002DFAD103239A
:103590006362FFF73BFFA562FFF760FF05B030BD38
:1035A0004843FF1F95FFFEF700C80040050001FFDC
:1035B00004E100E000E100E0FFFF00FFF0B585B0AE
:1035C0000700FEF7F9F9022305002D4C22681A4284
:1035D000FCD120230093009B5A1E0092002BFAD1AD
:1035E000284E3368002BFCDA0120FFF7F5FE002897
:1035F00003D01124200005B0F0BD234B236002232B
:1036000022681A42FCD120230193019B5A1E019289
:10361000002BFAD13368002BFCDA0120FFF7DCFE27
:103620000028E6D1194B1F60022322681A42FCD100
:1036300020230293029B5A1E0292002BFAD1336878
:10364000002BFCDA0120FFF7C7FE0028D1D1104B78
:103650002360022322681A42FCD120230393039B98
:103660005A1E0392002BFAD13368002BFCDA01209A
:10367000FFF7B2FE041EBCD12800FEF7B1F9B9E78E
:1036800090C8004000C8004001000006A8C80040E3
:103690000180000110B50020FFF790FF10BD000071
:1036A00010B5064B18705960FFF73CFF002113203E
:1036B000034AFFF72BFD002010BDC0464843FF1F03
:1036C0002535FF1FF0B5040085B003920291FEF787
:1036D00073F9882263035B0B52051A438023DB05D1
:1036E0009D6A8023274F0092BA68002601901B0331
:1036F0009A420CD9F82326001B041E401C4206D017
:103700008022214B52025E6219680A431A60002D22
:103710000BD100F045FC02221C4B1A608023DB0514
:103720005A62013A9A6200F0DBFB0023039A93424B
:1037300020D1002D0AD100F033FC144B03221D6070
:103740008023DB055A629D6200F0CAFB8023BA68C1
:103750001B039A4208D9002E06D000220A4B0C49BE
:103760005A621A680A401A600198FEF739F9002077
:1037700005B0F0BD009A0299D2181278CA540133EC
:10378000D4E7C0463C43FF1F00C8004000C00040D3
:10379000FFFFFEFFF0B587B0029103920400FEF731
:1037A0000BF9019000F0FCFB802302250122234E3F
:1037B000DB0535605D629A6200F092FB204F3B684A
:1037C0002B42FCD120230493049B5A1E0492002B0D
:1037D000FAD11C4D2B68002BFCDA0120FFF7FCFD11
:1037E000002802D0112007B0F0BD2000039A0299F2
:1037F00000F036FB022304003A681A42FCD1202371
:103800000593059B5A1E0592002BFAD12B68002BBD
:10381000FCDA0120FFF7E0FD051EE3D100F0C0FB5C
:1038200080230322DB0535605A629D6200F058FB5D
:103830000198FEF7D5F8E0B2D5E7C04600C00040D9
:1038400090C8004000C80040F0B5802489B0060050
:10385000FEF7B2F8E405A36A02250393029000F094
:103860009FFB0123304F3D606562A36200F038FB8F
:103870002E4C23682B42FCD120230593059B5A1E16
:103880000592002BFAD12A4D2B68002BFCDA01207F
:10389000FFF7A2FD002803D01124200009B0F0BDDD
:1038A000244B2360022322681A42FCD12023069372
:1038B000069B5A1E0692002BFAD12B68002BFCDACD
:1038C0000120FFF789FD021EE6D11B4B03211E607C
:1038D000030001900090202000F0CAFB0223226820
:1038E0001A42FCD120230793079B5A1E0792002BF4
:1038F000FAD12B68002BFCDA0320FFF76DFD041EC4
:10390000CAD100F04DFB80230322DB053C605A62E4
:103910009C6200F0E5FA039B002B01D1FFF776FDD6
:103920000298FEF75DF8B8E700C0004090C800407C
:1039300000C800400100000694C8004007B500021E
:1039400001910422000A01A9FFF724FF0EBD000027
:1039500073B5050005240B4AA3005B429B18196848
:103960006B46DE1D3000FFF787FA022804D133785A
:103970002B55013CEFD276BD052CFCD00128FAD1A5
:103980000230F8E7140900111F2807D8012380220C
:103990008340D20591680B43936070473F2808D855
:1039A0000123802220388340D20551690B435361A3
:1039B000F3E75F28F1D80123802240388340D20505
:1039C000116A0B431362E8E71F2807D80122802100
:1039D0008240C9058B6893438B6070473F2808D8A5
:1039E0000122802120388240C9054B6993434B61F5
:1039F000F3E75F28F1D80122802140388240C905D1
:103A00000B6A93430B62E8E71F2810D8802302005B
:103A1000DB05153A1968012A06D82022914319605E
:103A200019680A431A60704701228240F6E73F286E
:103A300011D880230200DB05353AD968032A06D85D
:103A400010229143D960D9680A43DA60EBE701227A
:103A500020388240F5E75F28E5D842238022181AF3
:103A6000413B8340D205516A99435162516A0B43ED
:103A70005362D8E710B50400012813D1A0221849D9
:103A800092050B685B015B0913430B60154B164AEB
:103A900019681140154A0A431A60402219680A43FE
:103AA0001A6010BD0028FCD101000A2000F0D0F8F7
:103AB00021000B2000F0CCF8C0220A4B92001968BC
:103AC0000A4340211A601A688A431A60B0220449E6
:103AD00012060B685B015B0913430B60E1E7C0460C
:103AE00014F000401CF000407F00FEFF80FD01004C
:103AF00072B6074A1368013313600422054B1A603B
:103B00000023054A13608022D2055360FEE7C046B9
:103B10007808FF1FC0F00040C4F0004005490B6862
:103B2000002B05D1044A0A6004490A60044A136064
:103B30007047C046140AFF1F841E0000380AFF1F8A
:103B4000C4F000400023034A1360034A1360034A91
:103B50001360704754F0004040F1004044F10040D1
:103B600002B4714649084900095649008E4402BC16
:103B70007047C04602B4714649084900095C4900D3
:103B80008E4402BC7047C04603B4714649084000E9
:103B90004900095E49008E4403BC704703B4714676
:103BA000490840004900095A49008E4403BC704747
:103BB00001B40248844601BC604700BF8512010081
:103BC00001B40248844601BC604700BFC9A9000097
:103BD00001B40248844601BC604700BFC95C0100D3
:103BE00001B40248844601BC604700BFCD4C0100CF
:103BF00001B40248844601BC604700BFD9B0000050
:103C000001B40248844601BC604700BFB70E000003
:103C100001B40248844601BC604700BF090E0000A1
:103C200001B40248844601BC604700BF85520100D0
:103C300001B40248844601BC604700BF8B520100BA
:103C400001B40248844601BC604700BFC1A5000022
:103C500001B40248844601BC604700BFCD9F0011FB
:103C600001B40248844601BC604700BF093401002A
:103C700001B40248844601BC604700BFEDA50000C6
:103C800001B40248844601BC604700BF2D6C0100AE
:103C900001B40248844601BC604700BF0134010002
:103CA00001B40248844601BC604700BF75F80000BB
:103CB00001B40248844601BC604700BF8D11010079
:103CC00001B40248844601BC604700BF5976010038
:103CD00001B40248844601BC604700BFA9D8000077
:103CE00001B40248844601BC604700BFB5B2000081
:103CF00001B40248844601BC604700BFE5120100E0
:103D000001B40248844601BC604700BF053401008D
:103D100001B40248844601BC604700BFD1AE000038
:103D200001B40248844601BC604700BFC1150100D0
:103D300001B40248844601BC604700BFE9F60000B8
:103D400001B40248844601BC604700BFC56D010054
:103D500001B40248844601BC604700BF69110100FC
:103D600001B40248844601BC604700BF116E0000E8
:103D700001B40248844601BC604700BF9D6A000050
:103D800001B40248844601BC604700BFDD0C01005D
:103D900001B40248844601BC604700BFE9D400007A
:103DA00001B40248844601BC604700BFD54401000D
:103DB00001B40248844601BC604700BF21440000B2
:103DC00001B40248844601BC604700BFBD5C0100ED
:103DD00001B40248844601BC604700BF8D820000E8
:103DE00001B40248844601BC604700BF49B20000EC
:103DF00001B40248844601BC604700BF0D52010077
:103E000001B40248844601BC604700BF21A90000FC
:103E100001B40248844601BC604700BFDD3F00009A
:103E200001B40248844601BC604700BFE90B0100B1
:103E300001B40248844601BC604700BF090E00007F
:103E400001B40248844601BC604700BFE94C010050
:103E500001B40248844601BC604700BFBD0B0100AD
:103E600001B40248844601BC604700BF957301005D
:103E700001B40248844601BC604700BFADAE0000FB
:103E800001B40248844601BC604700BF8937010085
:103E900001B40248844601BC604700BF85C10000F0
:103EA00001B40248844601BC604700BF8914010088
:103EB00001B40248844601BC604700BF791201008A
:103EC00001B40248844601BC604700BF016701009D
:103ED00001B40248844601BC604700BFC1660100CE
:103EE00001B40248844601BC604700BF9DA90000A0
:103EF00001B40248844601BC604700BF71B00000B5
:103F000001B40248844601BC604700BF01D70000ED
:103F100001B40248844601BC604700BFA1AF000065
:103F200001B40248844601BC604700BF53B9000099
:103F300001B40248844601BC604700BFED6801003F
:103F400001B40248844601BC604700BFCD0C0100AB
:103F500001B40248844601BC604700BF89440000A8
:103F600001B40248844601BC604700BFE917010064
:103F700001B40248844601BC604700BFED6B0100FC
:103F800001B40248844601BC604700BF6DF60000E2
:103F900001B40248844601BC604700BF156B0100B4
:103FA00001B40248844601BC604700BF75A9000007
:103FB00001B40248844601BC604700BFF5350100EA
:103FC00001B40248844601BC604700BFC1F700004D
:103FD00001B40248844601BC604700BFF9ED00000F
:103FE00001B40248844601BC604700BFF90D0100DE
:103FF00001B40248844601BC604700BFDD0A0100ED
:1040000001B40248844601BC604700BF6D0B01004B
:1040100001B40248844601BC604700BFE9270000A4
:1040200001B40248844601BC604700BFB35201009E
:1040300001B40248844601BC604700BFF935010065
:1040400001B40248844601BC604700BF61370100EB
:1040500001B40248844601BC604700BF3D710100C5
:1040600001B40248844601BC604700BF01890000DA
:1040700001B40248844601BC604700BF496D01009D
:1040800001B40248844601BC604700BF19FA000031
:1040900001B40248844601BC604700BF7997000024
:1040A00001B40248844601BC604700BF4DF90000DE
:1040B00001B40248844601BC604700BF75B30011DB
:1040C00001B40248844601BC604700BF016C010096
:1040D00001B40248844601BC604700BF51B80000EB
:1040E00002000000D2BC00110100000038BA00112B
:1040F00002000000CEBC0011010000002041FF1FA3
:104100000200000040BA0011010000001062FF1F11
:1041100002000000CCBC0011030000004461FF1F3E
:104120001200000002000000D2BC001101000000DB
:1041300084BA001102000000CEBC00110100000092
:1041400081BA0011020000008EBA001103000000C5
:10415000D761FF1F02000000CCBC0011030000006B
:10416000EC61FF1F02000000CEBC00110100000046
:1041700080BA0011020000008CBA00110300000098
:10418000AD61FF1F02000000CCBC00110300000065
:10419000CE61FF1F02000000D2BC00110100000030
:1041A000C4BA001102000000CEBC001101000000E2
:1041B0006942FF1F02000000D6BA00110100000092
:1041C000BEBA001102000000CEBC001101000000C8
:1041D0006842FF1F02000000D4BA00110100000075
:1041E000F461FF1F02000000CEBC001101000000BE
:1041F0006742FF1F02000000D2BA00110100000058
:10420000AEBA001102000000CEBC00110100000097
:104210006642FF1F02000000D0BA0011010000003A
:10422000A9BA001102000000CEBC0011010000007C
:104230006542FF1F02000000CEBA0011010000001D
:10424000A4BA001102000000CEBC00110100000061
:104250006442FF1F02000000CCBA00110100000000
:10426000A0BA001102020202020200000D4B00116E
:10427000D14A0011F4BA001190011D001800180075
:10428000FFFF07010203040506020106000000000B
:10429000000000000000000000000000000000001E
:1042A000000000000000000003000000000100000A
:1042B00000000111FFFF00005048593600000000C7
:1042C000000000000B000500F0000000B400002812
:1042D000002800283075A000A000A000A000000861
:1042E0000008E001F00010001000100010001000A5
:1042F000100050005000500010001000D0070000C7
:10430000000000000F0001000500307507001000DC
:10431000010081FF00000000FF000000B5710011E6
:10432000BD6F00114D6D0011FFFF0100FF00000087
:10433000D19B00114D9900116598001100000000FB
:104340000000000000000800040000003B0001081D
:104350005902E00188212800FF000000020000004F
:10436000D2BC00110100000098BD00110200000045
:10437000CEBC001101000000D943FF1F0200000065
:10438000CABC0011010000003068FF1F02000000DD
:10439000CEBC001101000000D843FF1F0200000046
:1043A000C8BC001101000000D643FF1F020000003E
:1043B000CEBC001101000000D443FF1F020000002A
:1043C000C6BC001101000000CC43FF1F18001800FC
:1043D0001D00900102000003020200000200000024
:1043E000D2BC001101000000ACBD001102000000B1
:1043F000CEBC0011010000001C44FF1F02000000A1
:10440000C4BC001100000000000000000200000019
:0E441000CCBC0011030000005068FF1F20FF0D
:040000051FFF184180
:00000001FF
